S01A0000666C6173686C6F616465725F6C6F616465722E73726563AF
S1130000000003201104000037940000379400001E
S1130010379400003794000037940000FCFD022060
S11300200000000000000000000000003794000001
S1130030379400000000000037940000379400005B
S1130040C9950000C9950000C9950000C995000034
S1130050C9950000C9950000C9950000C995000024
S1130060C9950000C9950000C9950000C995000014
S1130070C9950000C9950000C9950000C995000004
S1130400FFFFFFFFFFFFFFFFFFFFFFFFFE3DFFFFBB
S113041072B60E480E49886000220023002400258D
S113042000260027B846B946BA46BB46BC4609482A
S1130430854609488047094880470948804762B68D
S113044000200021074A9047FEE70000000000005A
S113045000ED00E0000003204995000039940000FD
S11304607F940000B104000072B60D4900200860BA
S1130470BFF36F8FBFF34F8F704780B548F6087294
S11304800FF23401074808F0ABFFFFF7EDFF064811
S113049080F3088880F309880448BDE802400047D7
S11304A008ED00E00000FF1FB8B7FF1F1104FF1F95
S11304B080B5FFF7E2FFFEE7B8B7FF1F1104FF1F87
S11304C0A70DFF1F2546FF1F2746FF1F2946FF1FB5
S11304D02B46FF1F2C06FF1F000000000000000039
S11304E000000000A70DFF1FA70DFF1F0000000064
S11304F0A70DFF1FA70DFF1F9F8EFF1F9F8EFF1FBE
S11305009F8EFF1F9F8EFF1F9F8EFF1F9F8EFF1FBB
S11305109F8EFF1F9F8EFF1F9F8EFF1F9F8EFF1FAB
S11305209F8EFF1F9F8EFF1F9F8EFF1F9F8EFF1F9B
S11305309F8EFF1F9F8EFF1F9F8EFF1F9F8EFF1F8B
S11305409F8EFF1F9F8EFF1F9F8EFF1F9F8EFF1F7B
S11305509F8EFF1F9F8EFF1F2365FF1F2765FF1FB1
S1130560CD47FF1FD147FF1F9F8EFF1F9F8EFF1F89
S1130570C767FF1FD767FF1FF567FF1F0B68FF1FC4
S11305801B68FF1F9F8EFF1F9F8EFF1F9F8EFF1FE5
S11305909F8EFF1F9F8EFF1F9F8EFF1F9F8EFF1F2B
S11305A09F8EFF1F9F8EFF1F9F8EFF1F9F8EFF1F1B
S11305B09F8EFF1F9F8EFF1F9F8EFF1F9F8EFF1F0B
S11305C09F8EFF1F9F8EFF1F9F8EFF1F0F8AFF1F8F
S11305D09F8EFF1F9F8EFF1F9F8EFF1F9F8EFF1FEB
S11305E09F8EFF1F9F8EFF1F9F8EFF1F8F24FF1F55
S11305F09F8EFF1F9F8EFF1F9F8EFF1FD547FF1FDC
S11306009F8EFF1F9F8EFF1F9F8EFF1F9F8EFF1FBA
S11306109F8EFF1F9F8EFF1F9F8EFF1F9F8EFF1FAA
S11306209F8EFF1F9F8EFF1F9F8EFF1F9F8EFF1F9A
S11306309F8EFF1F9F8EFF1F9F8EFF1F9F8EFF1F8A
S11308709F8EFF1F9F8EFF1FFFFFFFFFFFFFFFFFE6
S1130880FFFFFFFFFFFFFFFFFFFFFFFFFFFFFFFF74
S1130890FFFFFFFFFFFFFFFFFFFFFFFFFFFFFFFF64
S11308A0FFFFFFFFFFFFFFFFFFFFFFFFFFFFFFFF54
S11308B0FFFFFFFFFFFFFFFFFFFFFFFFFFFFFFFF44
S11308C0FFFFFFFFFE3DFFFF72B60E480E49886032
S11308D0002200230024002500260027B846B9463C
S11308E0BA46BB46BC46094885460948804709487C
S11308F080470948804762B600200021074A904794
S1130900FEE700000000FF1F00ED00E0B8B7FF1F86
S11309104D77FF1FAD40FF1FF340FF1FF339FF1F4B
S11309200000000000000000002A01D101207047EF
S1130930F0B41F46034603242340002B09D00424AB
S1130940E31A017001300824E141521E26D05B1ED7
S1130950F7D1042A1ADB13D0002F11D00C460D4610
S11309600E46102A02DB72C0103AFAE70C2A02DBA8
S113097032C00C3AFAE7082A02DB12C0083AFAE756
S1130980042A03DB01600430121FF9E7002A05D0B2
S1130990017001300824E141521EF7D1F0BC00205F
S11309A0704770476526FF1F000000008B26FF1F5D
S11309B0000000006927FF1FB728FF1F5727FF1FEC
S11309C0DB27FF1F8B29FF1F000000000000000031
S11309D000000000C526FF1F000000009F26FF1F27
S11309E0DB27FF1F9F29FF1F00000000212AFF1F94
S11309F0000000001B26FF1F00000000F926FF1F57
S1130A00000000000000000000000000412AFF1F59
S1130A1000000000672AFF1F00000000A32AFF1F38
S1130A20B728FF1F0F27FF1F000000000000000071
S1130A300000000000010246813AFF1FD53AFF1F63
S1130A4000000000F33AFF1F813BFF1F3D3DFF1FE5
S1130A506D3DFF1FCF3DFF1FDB3DFF1F633EFF1FAB
S1130A60693FFF1F00000000073CFF1FF93CFF1F08
S1130A704D3CFF1F00000000E73EFF1F0000000088
S1130A80000000000000000000000000570DFF1FE0
S1130A906D0DFF1F850DFF1F436F707972696768C5
S1130AA0742028632920323031332D3230313620FE
S1130AB0467265657363616C652053656D69636F28
S1130AC06E647563746F722C20496E632E20416CC2
S1130AD06C207269676874732072657365727665D9
S1130AE0642E0000EB04FF1F0000024BE005FF1F13
S1130AF0188FFF1F7C05FF1FD405FF1F0000000097
S1130B00798EFF1F838EFF1F8D8EFF1F0000000054
S1130B10000000009146FF1FD346FF1F2B47FF1F15
S1130B2000000000000000005F47FF1F01000000FC
S1130B301312FF1F0000000000000000312CFF1FF3
S1130B40612CFF1FA12CFF1F612DFF1F000000005F
S1130B509B2DFF1F2B65FF1F6B65FF1F1166FF1F7A
S1130B6000000000000000004D66FF1FE966FF1F43
S1130B706767FF1F8167FF1F00000000000000007F
S1130B80B367FF1F2745FF1FB143FF1FD943FF1F53
S1130B905544FF1F9144FF1F1544FF1F52656164B4
S1130BA0790D0A005472616E7366657272696E67BC
S1130BB00D0A0000537563636573730D0A0000002A
S1130BC04661696C7572650D0A000000EB3C904D3E
S1130BD05357494E342E310002010100022000FF18
S1130BE07FF080000100010001000000FF7F000091
S1130BF0000029313233344B696E657469732055B2
S1130C0053420000F0FFFFFFFFFFFFFFFFFFFFFF66
S1130C10FFFF000046534C204C6F6164657220084E
S1130C200000000000000000000000602C420000F2
S1130C3000000000412E0066007300650076000F7E
S1130C4000DA65006E0074007300640000000000A8
S1130C50FFFFFFFF46534556454E7E3120202012AC
S1130C60000000602C422C42000000602C42020074
S1130C700000000042650072005F0069006E000F12
S1130C8000A86400650078000000FFFFFFFF00007B
S1130C90FFFFFFFF012E006D006500740061000F6F
S1130CA000A864006100740061005F006E00000031
S1130CB0650076004D45544144417E312020202278
S1130CC0000000602C422C42000000602C42000016
S1130CD000000000412E0054007200610073000FF8
S1130CE000256800650073000000FFFFFFFF00009F
S1130CF0FFFFFFFF5452415348457E3120202022FC
S1130D00000000602C422C42000000602C420000D5
S1130D100000000042200049006E0066006F000FD2
S1130D20007272006D006100740069006F000000C1
S1130D306E00000001530079007300740065000F19
S1130D4000726D00200056006F006C0075000000FA
S1130D506D00650053595354454D7E3120202016B3
S1130D60000000602C422C42000000602C42030072
S1130D7000000000494E464F2020202054585420A3
S1130D80000000602C422C42000000602C42050050
S1130D90010000005354415455532020545854200A
S1130DA0000000602C422C42000000602C4206002F
S1130DB0010000002E20202020202020202020328E
S1130DC0000000602C422C42000000602C42020013
S1130DD0000000002E2E2020202020202020201083
S1130DE0000000602C422C42000000602C420000F5
S1130DF0000000004E4F5F4C4F4720202020202051
S1130E00080000602C422C42000000602C420000CC
S1130E10000000007B003300370032003000330054
S1130E204200460038002D004600440038003300DC
S1130E302D0034003300320031002D004100340015
S1130E40430034002D0039004100390041004200C4
S1130E5046003800460042004300460044007D003E
S1130E60000000002E2020202020202020202032DE
S1130E70000000602C422C42000000602C42030061
S1130E80000000002E2E20202020202020202010D2
S1130E90000000602C422C42000000602C42000044
S1130EA00000000042470075006900640000000F64
S1130EB000FFFFFFFFFFFFFFFFFFFFFFFFFF00003B
S1130EC0000000000149006E006400650078000F16
S1130ED000FF6500720056006F006C007500000092
S1130EE06D006500494E444558457E312020202040
S1130EF0000000602C422C42000000602C420400E0
S1130F004D0000005541FF1F5941FF1F6B41FF1F5A
S1130F10A941FF1F000000000000000001000000C4
S1130F2004000000D323FF1FB406FF1FC406FF1FE5
S1130F30200BFF1F02000000010000001724FF1F08
S1130F409C06FF1FAC06FF1F200BFF1F04000000C0
S1130F50010000004724FF1F5C06FF1F6C06FF1FF3
S1130F60200BFF1F10000000000000000000000024
S1130F703C0BFF1F000000004C0BFF1F0000000093
S1130F80000000000000000000000000000000005D
S1130F9000000000CD70FF1F0B71FF1F2172FF1FA7
S1130FA0F972FF1F1C9BFF1F0531FF1F172FFF1F27
S1130FB00931FF1F1331FF1F1B30FF1F1D31FF1F9E
S1130FC02531FF1F172FFF1F2931FF1F3331FF1F4B
S1130FD01B30FF1F3D31FF1FFD73FF1F0374FF1FF5
S1130FE06B74FF1F0975FF1F0174FF1F1575FF1F29
S1130FF0DD73FF1F5D86FF1F5B87FF1F4B88FF1F8D
S11310008188FF1FB788FF1FDB88FF1F6389FF1FCD
S1131010F789FF1F078AFF1F0B8AFF1F00000000CC
S11310202DE9FF4B0C46434E0178DFF80CB13170CB
S113103090464178717001258178B170C178F17062
S113104001793171417971718179B171C179F1712C
S113105000EBC5020BEBC50113780B706D1C5378C4
S11310604B70062D00F06AF8F2DB4FF005090525F8
S113107030788DF8000009EB890170788DF8010053
S11310806918B0788DF802000BEBC507F0788DF87D
S113109003006A4630798DF804006D1E00F074F880
S11310A048408DF80700414600F085F800F0C6F886
S11310B09DF800003070012D9DF8010070709DF8BE
S11310C00200B07000F068F8F07100F044F8CFDA74
S11310D0B9F10109CBD500F088F80BEBC00204EBA1
S11310E0C00113780B70401C53784B70062800F035
S11310F025F8F2DB2078A62804BF6078A62812D150
S1131100A078A62804BFE078A6280CD12079A628C8
S113111004BF6079A62806D1A079A62802BFE07989
S1131120A628002001D04FF0FF3004B0BDE8F08BBA
S1131130000000004899FF1F5099FF1F93788B709F
S1131140D378CB7013790B7153794B7193798B717D
S1131150D279CA7170479DF8080038709DF809006B
S113116078709DF80A00B8709DF80B00F8709DF82F
S11311700C0038719DF80D0078719DF80E00B8715F
S11311809DF80F00F871704770798DF80500B079FB
S11311908DF80600F07970479DF80300F0709DF813
S11311A0040030719DF8050070719DF80600B0715F
S11311B09DF80700704738788DF8080078788DF826
S11311C00900B8788DF80A00F8788DF80B003879A2
S11311D08DF80C0078798DF80D00B8798DF80E0033
S11311E0F8798DF80F006846704730782070707871
S11311F06070B078A070F078E07030792071707908
S11312006071B079A071F079E0710120704710B578
S1131210044600F05CF820B12046BDE8104000F020
S11312209CB810BD70B500F015F830B132462946AF
S11312302046BDE8704000F096B870BD70B500F06F
S113124009F830B1324629462046BDE8704000F026
S11312509CB870BD04460D46164600F038B8FEE74B
S11312600120704730B585B000F029F8D0B12C4C7E
S1131270A06800688047A0680069D0F88C1011F15C
S1131280010F08BF4FF482616A46002000F007F99D
S1131290694600220023002400253CC110B9214ADC
S11312A00121117005B030BD80B51E48007810B121
S11312B0002000F033F9002002BD00F0EBBD1A4815
S11312C00068000E10F00F0018BF01207047164888
S11312D00068000E00F00F00012816BF022801204C
S11312E000207047114800687047104908600C4995
S11312F0896809694865704710B582B000228DF885
S113130000200A46064C014604F120002469646C5E
S11313106B46A0479DF8000000B1012016BD0000F7
S1131320188FFF1FB2A7FF1F248004406C8FFF1F7C
S113133010B5002150F8212002F47F431B02140A47
S113134043EA026304F47F44234343EA126240F80D
S11313502120491C0429EDD310BD3248016841F411
S1131360003101607047F8B500F025F800F021F86D
S113137000F02AF82C4800F033F800F01AF8B442D0
S11313801CBF3046FFF7D4FF10E0F8B500F013F8A7
S113139000F00FF800F018F8244800F021F800F0ED
S11313A008F8B4421CBF3046FFF7C2FF0020386182
S11313B0F1BD2046BCE704461D4F4FF0FF303864B2
S11313C00D4616462846B3E71A482968016069683D
S11313D04160A9688160E968C1601020B860704705
S11313E0386010203861B86C40F48030B8642168EB
S11313F01148016061680160A1680160E1680160F1
S1131400B96CC903FCD50169316001697160016976
S1131410B1600069F060B86C40F48030B86428466C
S113142086E700002C8004400D0210000C0210001E
S113143000100D4000120D40E0170D402DE9F04161
S113144096B004460D46164600F078FD8046002707
S11314501CE0324603A92846FFF7E2FDA0B901A823
S113146000F08AFD202205A901A800F08BFD694641
S113147001A800F09DFD00980E99884204D105AAA8
S11314803946204600F05EFD40357F1C4745E0D3D9
S1131490482103A800F0A2FF16B0BDE8F081F8B51A
S11314A014460FF28C021C4E52F820504FF48072F6
S11314B0304600F097FF06F5807710222146384623
S11314C000F090FF3846FFF7A2FE284600F020FD0A
S11314D040F2F514C0B9284600F02BFDC8B93A46CD
S11314E031462846FFF7AAFF284600F015FD284696
S11314F000F017FD0028284602D100F015FD08E091
S113150000F012FD0020F2BD022802D14FF4FA705F
S1131510F2BD2046F2BD0000D899FF1F80B50FF23E
S1131520100151F8200000F0F7FC002002BD00007B
S113153000AC0D40DFF87409016841F440610160BA
S1131540016811F4406FFBD17047DFF864190A6831
S1131550904202D24FF0D04070474A68904201D284
S113156008687047CA68904201D248687047CA68E0
S1131570904234BF88684FF0FF3070472DE9F04146
S113158000F07DF8DFF82C49DFF82C59DFF82C79CE
S11315904FF0006000F06DFA00F071F82E683868C2
S11315A0C0B1D7F80C8018F1010F04D03046FFF712
S11315B0CCFF404428604FF01060206000F013F826
S11315C0D7F8108018F1010F04D03046FFF7BDFFA3
S11315D0404428604FF08070206000F004F83868C0
S11315E000B12E6040E2F8B54FF47A7000F06EFF5F
S11315F004460D4600F060FF4FF47A72A2FB0467C4
S113160002FB0577841941EB070500F055FF8D4275
S113161005D828BF844202D240F29910F2BDDFF807
S1131620A0080068C007F0D40020F2BDDFF89418C9
S1131630D1F8D021022A00D2704710B5DFF86C48E7
S1131640226842F480420128226011D1D1F8D001ED
S1131650A0B12168090E491C4843112828BF102055
S113166021680902090A401E41EA0060206005E081
S1131670022803D1486CC0B200F058FF20E0DFF824
S113168048180A6840F2011002430A600A680242DC
S1131690FCD1704710B5DFF81448206820F480406E
S11316A02060206840F0030020600A2000F017FF4B
S11316B0206840F48040206020688008800020601A
S11316C0206820F48040206010BDDFF80028DFF897
S11316D0003850B1012811D0022812D0032813D0A9
S11316E0042813D0102813D014E01878002814BF4D
S11316F0002040F295100860002070474FF0D04061
S1131700F9E75868800AF6E71068F4E75068F2E7EA
S11317105868F0E7042070472DE9F04FDFF8A4A7DC
S11317200AF5E67787B0386800B1012004900024F8
S11317304FF47A7000F0CAFE81460498A0468B46A6
S113174050B100F0B9FE04463868A9FB00230BFB36
S11317500033CDE902238846DAF84810DFF85457FD
S1131760DFF854670120884001900020009004981D
S113177038B100F0A1FE00F057F835D301D89042FB
S113178032D3FFF7D7FEFFF77AFF3468B86888B121
S1131790D7F8108018F1010F04D02046FFF7D5FECA
S11317A0404430604FF030602860FFF71CFF002891
S11317B037D134604FF040702860FFF714FF80BBCE
S11317C000F07AFE04464FF47A70A0FB092300FB74
S11317D00B33CDE90223884600F06EFE00F024F8B6
S11317E005D828BF904202D240F2971019E0F06861
S11317F010F4F85FF0D0DFF8DC0600680090306E7B
S113180040F480303066DAF84800C003009804D50C
S11318100199C0430842AAD102E001990842A6D125
S1131820002007B0BDE8F08F021B61EB0803DDE97F
S113183002019942704750B5DFF8882683B0526B95
S1131840A0F1D0400C46B0EB420FDFF8641604D28E
S11318504FF0D0400090486802E008680090886823
S1131860019000265DF82600DFF84C160860200081
S113187001D0A04718B9761C022EF3D300205EBD18
S11318802DE9F04FDFF83C6681B0D6F8C4A11418F6
S11318908046F06D89464AF08065002718B145F40A
S11318A0803500E0D044A04580F07D800120FFF722
S11318B0BDFEDFF80076C7F8F880F06D10B9FFF7C9
S11318C05DFE06E0DFF810164046FFF7B4FFC7F8E8
S11318D0F880D6F8D40198B1FFF7D1FED6F8E8B174
S11318E01BF1010F05D04046FFF72FFE5844C7F8FF
S11318F0F8004FF020603860FFF775FEC7F8F880F5
S1131900FFF7BDFEFFF716FED7F8580140F0006060
S1131910C7F85801EFF3108072B6102159F8042B60
S1131920C7F84C21491EF9D10321C7F850113D6075
S1131930AAF14001890810E059F8042BC7F84C219A
S1131940091F59F8042BC7F84C2159F8042BC7F880
S11319504C2159F8042BC7F84C210129C0F2088006
S1131960D7F854219201E7D4D7F858215201F7D57A
S113197080F31088FFF737FE0220FFF757FED7F8F1
S11319805801400102D54FF4CC770CE0F06D10B94A
S1131990FFF7C2FE04E0DFF844154046FFF74BFFB3
S11319A007003FF47FAFFFF775FE384601B0BDE88E
S11319B0F08F00002DE9F041804600204FF0D04523
S11319C00026DFF8007506E00024032E0AD8DFE8BD
S11319D006F0020406087C6B04E0BC6B02E0FC6BBE
S11319E000E03C6C2CB1DFF8D00405602846C04709
S11319F018B96519761C042EE6D3BDE8F0812DE9EB
S1131A00F04105460120FFF711FEFFF7B7FDDFF8AF
S1131A10AC74DFF8A0443868E8B1D7F81880DFF870
S1131A20986418F1010F04D02846FFF78EFD404456
S1131A303060FFF724FE00F01AF83560786808B1CA
S1131A40FFF79CFDFF6917F1010F04D02846FFF74B
S1131A507CFD38183060FFF712FE4FF0007000F084
S1131A6008F80220FFF7E2FD0020BDE8F0814FF006
S1131A70C0602060B7E54FE610B5DFF86404FFF7F7
S1131A8099FFDFF86004FFF795FF0446FFF702FEB5
S1131A90204610BD2DE9F04105460120FFF7C6FDA3
S1131AA0DFF81464DFF81474DFF808443560FFF7D6
S1131AB065FD386890B1D7F8188018F1010F04D08B
S1131AC02846FFF742FD40443060FFF7D8FDFFF79A
S1131AD0CEFF3560786808B1FFF750FDFFF7CFFD02
S1131AE04FF0E060FFF7C5FF0220FFF79FFDFFF70F
S1131AF013FE0446FFF7CEFD2046BDE8F08170B525
S1131B00DFF8C043E16DB9B1626BDFF8DC63A0F1CB
S1131B10D0414D08B1EB420F05F1D04005D2FFF79B
S1131B20B9FF60B93068281806E0FFF7B3FF30B991
S1131B307068616B2818401ABDE87040AAE770BD50
S1131B40F8B5DFF86813DFF8A423CA610A6822F045
S1131B50E0020A6000F10C02936C1BB10B6843F0C5
S1131B6080030B60DFF85C53D66C012405F5BA736F
S1131B703EB30E6846F040060E6000F5D470066869
S1131B801EB10E6846F020060E601E6B0EB141F2C7
S1131B9001048668C768B6023F0406F4406607F489
S1131BA07C173E43076912683F0607F07C573E43A3
S1131BB0344332B1406800280CBF44F4007444F448
S1131BC0807405F11000C26B032A08BF44F400447A
S1131BD09A6A0AB144F48044DA6A0AB144F40054BB
S1131BE04C62856DC46DA4016D0104F0400405F0E0
S1131BF020052C43056EBE4A2D0405F4E0252C4334
S1131C005460C46C240404F480340C6284691B782A
S1131C10240403F00F0304F4803423431360C269E3
S1131C2090F82030120202F4706203F00F031A439A
S1131C3003681B0403F440331A43CA60406BC0B208
S1131C4000F074FC0020F2BD2DE9F84F8146FFF747
S1131C50CAFCA84F386840F080603860484600F0FD
S1131C6077FC002850D1974E9149706B984C00F145
S1131C70D04008604FF0D048B26B10184860F26B47
S1131C8010188860326C1018C8600021A0F1D04090
S1131C9060600091404609F13401042251F8043B8C
S1131CA013B1056800951818521EF7D10098FFF774
S1131CB0F1FC606848B1F06D48B1706BF16B88421B
S1131CC002BFB06B316C884201D004207FE08A49A6
S1131CD08A4A0A6002234B600020002306EB830437
S1131CE0874D646F45F82040401C5B1C402BF5D3A6
S1131CF00A60012048606D4E306840F480403060D6
S1131D004846FFF71DFF20B1396821F08061396032
S1131D105DE03068684F20F480403060386940F4FA
S1131D2080703861D9F8780190B309F134004446E1
S1131D30009004250098001D0090001F006828B33F
S1131D403C60041909F5BC704068F8B14FF0000A12
S1131D5009EB8A0000F5BE7BDBF80000B0B1FFF7A9
S1131D600DFCFFF78CFCFFF7E5FBDBF8100000F03F
S1131D7030F8DBF80000B060FFF735FCFFF7CCFC6F
S1131D8020B90AF1010ABAF1040FE1D36D1ED1D1D1
S1131D9009F11C042068C8B109F13409042559F873
S1131DA0040B88B1C7F800808044FFF7E7FBFFF716
S1131DB066FCFFF7BFFB606800F00BF8A068B0603A
S1131DC0FFF711FCFFF7A8FC6D1EE8D10020BDE869
S1131DD0F28F786500207865786578657047F8B586
S1131DE0050018BF15F0030044D1394C00202070C1
S1131DF0284600F0ADFB3F48016841F08061016076
S1131E002A48016841F4804101600121416201686E
S1131E100902090A41F0807101603A49C1610E2149
S1131E20016141618161016841F00C010160016857
S1131E3021F480410160FDB9334F4FF0D04635465F
S1131E40306800900098FFF725FC3068B8420CD049
S1131E5029482A490160022242602C4A026141F663
S1131E6004424261016001214160FFF713FC3068C4
S1131E70B84201D00420F2BD124E4FF4007229463C
S1131E80304600F0BFFA3046FFF7DEFE08B9012104
S1131E902170F2BD0E480078704780B50C48007878
S1131EA008B1FFF7F7FB002002BD000000A00D40C1
S1131EB080A10D4008A00D4000A10D40AC9DFF1F66
S1131EC05CA10D40D89BFF1F6CA10D409C9DFF1F82
S1131ED0D89DFF1F00A20D40C510FF1F6112FF1FF8
S1131EE04715FF1FBF15FF1F84A10D400040008050
S1131EF004A10D402C80044000A30D40F05AF05A78
S1131F0010A30D40000800806B7163661304200861
S1131F104068C0F381007047016841F000410160EE
S1131F2070470068C00F7047016841F0800101608C
S1131F3070470068C00900F0010070474068C0F3B2
S1131F400310704700EB811000F580701168016088
S1131F505168416091688160D168C1601169016113
S1131F605169416191698161D169C16170470268B8
S1131F70531C0360117070474FF0FF310160002162
S1131F804160704730B544680368141944600FF227
S1131F904C0407E011F8015B85EA136554F82550F9
S1131FA085EA032315466A1E002DF3D1036030BD74
S1131FB030B54368026813F0030F0CD003F0030339
S1131FC0C3F104030FF21404150E54F825505B1EDC
S1131FD085EA0222F8D102600A6030BD00000000E8
S1131FE0B71DC1046E3B8209D926430DDC76041368
S1131FF06B6BC517B24D861A0550471EB8ED0826FF
S11320000FF0C922D6D68A2F61CB4B2B649B0C359B
S1132010D386CD310AA08E3CBDBD4F3870DB114C48
S1132020C7C6D0481EE09345A9FD5241ACAD155F2B
S11320301BB0D45BC2969756758B5652C836196A34
S11320407F2BD86EA60D9B6311105A6714401D791F
S1132050A35DDC7D7A7B9F70CD665E74E0B62398C9
S113206057ABE29C8E8DA191399060953CC0278B33
S11320708BDDE68F52FBA582E5E66486585B2BBEBA
S1132080EF46EABA3660A9B7817D68B3842D2FADD7
S11320903330EEA9EA16ADA45D0B6CA0906D32D47A
S11320A02770F3D0FE56B0DD494B71D94C1B36C7AF
S11320B0FB06F7C32220B4CE953D75CA28803AF2B8
S11320C09F9DFBF646BBB8FBF1A679FFF4F63EE113
S11320D043EBFFE59ACDBCE82DD07DEC77708634D8
S11320E0C06D4730194B043DAE56C539AB06822747
S11320F01C1B4323C53D002E7220C12ACF9D8E1286
S113210078804F16A1A60C1B16BBCD1F13EB8A01BA
S1132110A4F64B057DD00808CACDC90C07AB977847
S1132120B0B6567C69901571DE8DD475DBDD936B8A
S11321306CC0526FB5E6116202FBD066BF469F5E6B
S1132140085B5E5AD17D1D576660DC5363309B4D3E
S1132150D42D5A490D0B1944BA16D84097C6A5ACCC
S113216020DB64A8F9FD27A54EE0E6A14BB0A1BF92
S1132170FCAD60BB258B23B69296E2B22F2BAD8AC1
S113218098366C8E41102F83F60DEE87F35DA99976
S11321904440689D9D662B902A7BEA94E71DB4E039
S11321A0500075E4892636E93E3BF7ED3B6BB0F30E
S11321B08C7671F7555032FAE24DF3FE5FF0BCC6EF
S11321C0E8ED7DC231CB3ECF86D6FFCB8386B8D532
S11321D0349B79D1EDBD3ADC5AA0FBD8EEE00C6912
S11321E059FDCD6D80DB8E6037C64F643296087A18
S11321F0858BC97E5CAD8A73EBB04B77560D044F6B
S1132200E110C54B383686468F2B47428A7B005CEB
S11322103D66C158E4408255535D43519E3B1D25A4
S11322202926DC21F0009F2C471D5E28424D1936DB
S1132230F550D8322C769B3F9B6B5A3B26D6150320
S113224091CBD40748ED970AFFF0560EFAA011106F
S11322504DBDD014949B93192386521D0E562FF115
S1132260B94BEEF5606DADF8D7706CFCD2202BE263
S1132270653DEAE6BC1BA9EB0B0668EFB6BB27D7A6
S113228001A6E6D3D880A5DE6F9D64DA6ACD23C4A7
S1132290DDD0E2C004F6A1CDB3EB60C97E8D3EBDB6
S11322A0C990FFB910B6BCB4A7AB7DB0A2FB3AAEDF
S11322B015E6FBAACCC0B8A77BDD79A3C660369B24
S11322C0717DF79FA85BB4921F4675961A163288E3
S11322D0AD0BF38C742DB081C330718599908A5DF8
S11322E02E8D4B59F7AB085440B6C95045E68E4E77
S11322F0F2FB4F4A2BDD0C479CC0CD43217D827BF2
S11323009660437F4F460072F85BC176FD0B86688A
S11323104A16476C93300461242DC565E94B9B1123
S11323205E565A1587701918306DD81C353D9F02BA
S113233082205E065B061D0BEC1BDC0F51A6933757
S1132340E6BB52333F9D113E8880D03A8DD097240E
S11323503ACD5620E3EB152D54F6D4297926A9C598
S1132360CE3B68C1171D2BCCA000EAC8A550ADD642
S1132370124D6CD2CB6B2FDF7C76EEDBC1CBA1E3AD
S113238076D660E7AFF023EA18EDE2EE1DBDA5F0C6
S1132390AAA064F4738627F9C49BE6FD09FDB889F5
S11323A0BEE0798D67C63A80D0DBFB84D58BBC9ABE
S11323B062967D9EBBB03E930CADFF97B110B0AF5B
S11323C0060D71ABDF2B32A66836F3A26D66B4BC82
S11323D0DA7B75B8035D36B5B440F7B1002200F07E
S11323E08FB9000062B38B0708D0521E11F8013B6D
S11323F000F8013B00F024808B07F6D1830740F0FE
S1132400208000BF103A07D330B4B1E83810103A36
S1132410A0E83810F9D230BC530724BFB1E8081043
S1132420A0E8081044BF51F8043B40F8043BD2072D
S113243024BF31F8022B20F8022B44BF0B78037021
S11324407047083A07D3B1E80810083A40F8043B4B
S113245040F804CBF7D25307E4E7000080B52B48DB
S1132460016841F4000101600020294908604FF02F
S1132470FF3128480161002282610122C261826920
S113248042F004028261826942F0010282610160C9
S11324900121C160816000F0FAF8C0001E49B0FB60
S11324A0F1F000B901201D49086001BD1848016818
S11324B041F002010160704710B5194B19691A689F
S11324C01C68A242FAD3D043C94310BD134909681A
S11324D0A1FB0001C00840EA4170C908704738B543
S11324E00446FFF7E9FF0D4A1268A2FB0423D20851
S11324F042EA4372141841EBD305FFF7DDFFA9420A
S1132500FBD301D8A042F8D331BD00003C80044085
S1132510007003400071034040420F00009BFF1F06
S11325200471034000F0B3B87047000007490A681B
S11325301202120A012804D0022804D042F0407288
S113254001E042F080720A607047000000A00D4074
S1132550F0B501250024002600F134024FF4A063F5
S1132560504908B9012615E09769042F0BD30020C0
S113257051F8202022F4E06241F82020401C0E286B
S1132580F6D30420F0BD176807B90025976807B192
S113259001242DB34B608B600B614B6186BB566885
S11325A04FF4E06506B1CD619669022E12BF032E89
S11325B00B60CB609669032E0FD10B628B624B626A
S11325C000F5CE708B61066806B1CB614668002EBB
S11325D01FBF0B63006800284B63506A00B1CD62D3
S11325E074B1CB610B628B62CB629069022804BF29
S11325F04B628B61D06800B14B63506A00B10B63CE
S11326000020F0BD2848294A0168490849000160B2
S11326102748416B41F478514163016821F04061DE
S113262011430160704710B51F48214C016841F007
S113263001010160FFF72EFC0028606B14BF20F439
S1132640F05020F4785060631A4801684900490842
S11326500160206818490840206010BD14480168D2
S113266041F4E0210160016B41F4802101631148D0
S1132670016841F0004101601048017841F0800197
S11326800170017941F002010171012070470C4889
S11326900C4A016800681268090F491CC0F3036002
S11326A0514321E000D0044000D000400000030466
S11326B00480044000700440FFFFF8F34021074009
S11326C0448004405C90FF1F0148024A04E000BFBC
S11326D064800440006CDC020168006801F00101C0
S11326E0491CC0F342005143401CB1FBF0F0704759
S11326F0002070477047000062F30F2262F31F420C
S113270000B500BF130096469446103928BFA0E8D0
S11327100C50FAD85FEA417C28BF0CC048BF40F88F
S1132720042BC90728BF20F8022B48BF00F8012B4F
S113273000BD000038B504463D4D0020C5E9000049
S1132740C5E90200C5E90400286268623948FFF758
S1132750BDFEC5E906012046BDE834400FF255012F
S113276000F002B900F012B970B5314D0C46296A77
S1132770072904BF696A88421AD1FFF7D3FEC0EB68
S11327800016D5E90001D5E902231018B6FBF0F0D4
S11327900A2148434FF49661B0FBF1F0401D0A2131
S11327A0B0FBF1F04FF4966148432060002070BD07
S11327B0012070BD2DE9F8430646FFF77DFE1C4F4E
S11327C00446386AD7E904598846421CD7E9060109
S11327D0651B68EB0909494502D82CBFA8420122B0
S11327E0012A3A6206D0042A08D0052A0ED0072A04
S11327F00FD018E0C7E900487E6214E0D7E9000171
S1132800201A68EB0101C7E900010CE0C7E902489E
S113281009E0D7E90201201A68EB0101C7E90201C6
S1132820304600F0B3F8C7E90448BDE8F18300007E
S11328302099FF1F803801000901002806D55F4A4E
S113284000F00F00801800F8041C70475C4A8154A3
S1132850704750F82130120423F4702302F47022DC
S11328601A430FE050F82100C0F30060704706E0FF
S1132870120202F4E06242F0200203E000BF1202FE
S113288002F4E06240F821207047042800D0704729
S113289010B54C4C19B102290ED004D310BD002040
S11328A0A063E06310BD4FF48070A06346480168E4
S11328B021F48041016010BD03220E212046FFF760
S11328C0D6FF2046BDE8104003220F21CFE70128A0
S11328D000D0704710B53B4C11B1022904D010BD93
S11328E00020A062E06210BD02220B212046FFF707
S11328F0BFFF2046BDE8104002220A21B8E70128A4
S113290000D0704710B5314C11B1022906D010BD6A
S1132910002020616061A061E06110BD07220421F4
S11329202046FFF7ABFF072205212046FFF7A6FF4D
S1132930072206212046FFF7A1FF2046BDE81040EC
S1132940072207219AE780B50E211E48FFF78AFF68
S113295048B11F480169080005D0042088471D4973
S11329604FF0FF30086001BD10B504280C460CD1AF
S113297001213D20FFF760FF17494FF00050086028
S11329800A2200F016F81248046110BD042800D091
S1132990704780B511494FF00050086000213D2078
S11329A0FFF74AFF002200F004F8094900200861FB
S11329B001BD0E2103484CE70000000018ED00E0C3
S11329C000E400E000B0044094F00F4000C0044074
S11329D0089BFF1FA0B0044004E100E084E100E094
S11329E0DFF89016C968C9680020086070472DE9AF
S11329F0F041DFF8805682B0E86900248DF8014088
S1132A004669002E62D0E968C9680A68012A4CD078
S1132A1001F1080274680023091DA04704001FBFC8
S1132A2042F21270844242F2137084424ED1E8683A
S1132A30C168D1F80880B8F1000F47D04E683778E4
S1132A4037B1132F04DA806800EBC700083800E0C0
S1132A500020086200281CBF006800281CD02A69D6
S1132A609269694605F120009047040016D19DF84B
S1132A70000040B14FF4E750791EC840C00758BF6A
S1132A8042F211740AD5EA68D268126A12684146A1
S1132A9030469047002406E042F21074394620463E
S1132AA000F070FA94B901200DE0086A48B1416859
S1132AB0080003D00DF10100884704460CB1002042
S1132AC001E09DF80100E968C96808602046BDE896
S1132AD0F68180B50178002000F054FADFF89405FF
S1132AE0C069416909698847022000F0CBFABFF345
S1132AF04F8FDFF88405DFF88425016801F4E06175
S1132B0011430160BFF34F8F00BFFDE7DFF8640599
S1132B10C068C06814210C30FFF760BC10B50446CF
S1132B20606810B1012803D005E000F0ADFB03E0BC
S1132B3000F01DFD00E00420FFE72178BDE810400F
S1132B4020E210B5DFF82C25126852690446A1680A
S1132B5060689047F1E710B500F06EF8DFF81405EF
S1132B60C068C0686168016108210177002021788C
S1132B7000F008FABDE8104000F087BF30B583B01C
S1132B80DFF8F044A5680021019100916B4681684B
S1132B904068AD6801AAC9B2C0B2A847E268D26869
S1132BA00021116100998A08019900F0FFF937BDED
S1132BB010B5DFF8C0249268D26804466068A16842
S1132BC0C0B29047B9E770B504466068A5680128AB
S1132BD005F2FF1607D1284601F058F818B130461F
S1132BE001F054F808B904250CE02846FFF7F7F87B
S1132BF00500DFF8806402D1306800688047B0685F
S1132C000069456528462178BDE87040BAE110B5F1
S1132C1000F012F800F012F80421017700208CE78C
S1132C2010B500F009F800F009F80321017700203D
S1132C30A168BDE81040D0E1044667E7DFF834043A
S1132C40C068C068A168016161684161704738B5B6
S1132C5000F088F8002141610161007F042804D15B
S1132C6028680069804704B90446E868C068017FA1
S1132C70204600F087F942F21270844208D1E868D5
S1132C80C068007F082804BFBDE8314000F074BF6D
S1132C9031BD2DE9FC4100F065F8016921B900203E
S1132CA02070FFF7D4FF5AE00121217006694769BB
S1132CB0002000900123E869D0F814C0DCF804C0B7
S1132CC06A4601A9E0475FEA000805D0E86941695E
S1132CD0C9688847404603E0009830B942F2127050
S1132CE0FFF7B5FF002020703AE0B04288BF3046BD
S1132CF00090E868C068017F082913D10199C16078
S1132D00009981610198009900F001FF804642F228
S1132D107D7080451CBF42F2747080450BD14FF02A
S1132D20000808E02B68019A00999B683846984788
S1132D3080460098C7190098361A06D0B8F1000FDB
S1132D4009D0E8694169C96888474046FFF77FFFB1
S1132D500020207003E0E868C06806614761002035
S1132D60BDE8F681C34D0446E868C06870472DE9A4
S1132D70F047C04D8AB00446E868C068016921B9CB
S1132D8000202070FFF763FF57E0012121700669DE
S1132D904769C168027F212E2CBF4FF02008B0463E
S1132DA0A9B1424601A8FFF71DFBE869D0F814C099
S1132DB0DCF808C00123424601A9E047A6EB080657
S1132DC006B1B0B3FFF743FF0020207035E0032ABB
S1132DD008EB070907D12B685B6801AA414638460E
S1132DE09847824614E0102A18BF4F46DDD190F868
S1132DF01DA001F090F839462F69CDF800A0434694
S1132E00FF6B01AA05F12000B847824601F089F85A
S1132E10BAF1000F4F46C8D0E8694569AD6801238F
S1132E20002201A9A8475046FFF711FF0020207097
S1132E3004E0E868C0680661476100200AB0BDE8A4
S1132E40F08710B58B4B1B68DB680446E268A16809
S1132E506068984771E62DE9F0410546884C6E6834
S1132E60D5F80880E8688349206000274968103154
S1132E7030B10A68904223BF4968491C8142042743
S1132E80304600F003FF00B90427FEF716FA40B1FC
S1132E90FFF703F8FEF7E6F908B140F2F717FEF77B
S1132EA024FA2978384600F06DF89FB9666000204E
S1132EB000F0E8F82068C4F8088018B180F30888A6
S1132EC080F30988616840468847BDE8F0410020E6
S1132ED000F0D8B8BDE8F08138B50446606800F069
S1132EE0D5FE08B9042005E06568012000F0CAF8A1
S1132EF0A068A84721780FE038B55E4D044601F07C
S1132F000AF800F024F86D6B04F10C02A84705469A
S1132F1001F007F821782846BDE8344032E030B5A6
S1132F2083B0044668460021002206C0514D00F0DB
S1132F30F2FF00F00CF8AD6B6A46A847054600F0B6
S1132F40F0FFA2686946284600F04BF837BD05F14A
S1132F5020002D69A3686168704710B5FFF76CFE07
S1132F604448C168C968A2680A6162684A6110225B
S1132F700A77C068C068E16841770020A168BDE8AD
S1132F8010405BE010B584B0A02201908DF80020C1
S1132F90002200F06AF88DF80220029102228DF8D6
S1132FA0032000234469A4680C225BE010B588B0B8
S1132FB0A72300F03AF80020531C8DF8033006E0F4
S1132FC06C4651F8203004EB8004401CA36090420E
S1132FD0F6D300F021F800231AE010B584B0A32240
S1132FE02FE010B588B0AF2300F01FF802238DF84E
S1132FF0033040B99008801C8DF80300029203A8A6
S1133000FFF700FA01E000200290002300F004F82A
S11330106946A04708B010BD1648C0699DF8031062
S11330204469A46889000A1D70478DF80030019036
S113303000238DF801308DF80230704710B584B04C
S1133040B0228DF800200190012200F00EF80291C8
S113305000228DF80220002302228DF803200C2286
S11330604469A4686946A0471FBD0248C0698DF839
S113307001207047188FFF1F0CED00E00400FA05D3
S1133080A499FF1F70B50446022C04D0002001F05F
S113309002FA012C0ED00026114D06E04019C16839
S11330A089680A0018BF8847761C18207043415964
S11330B00029F3D174B900F02EFFFFF7F7F901F0FE
S11330C074FA0849002008600120FFF72DFAFFF781
S11330D0AAFA62B6BFF36F8FBFF34F8F70BD00BF04
S11330E0640AFF1F08ED00E038B5934D2B696C6846
S11330F0DB6A2246042105F1200098472B69DB6A2C
S11331006A46012105F120009847206800990818B3
S1133110401E6060002032BDF8B5874F0446786BCE
S11331200D464042164600EA0401621AAA185242A9
S11331301040424207F120003F697F6C6B46B8475C
S113314048B99DF8000008B16C20F2BD324629460A
S1133150204601F05DFAF2BD2DE9F04389B09146B5
S113316004460F4603AA00F0CEF8002846D1BE0854
S1133170B600BF1B4FF0FF300690079005D03A46CB
S113318006EB090106A8FFF72DF906EB04086A4DC2
S113319056B1D5F810C0DCF814C033464A4621466F
S11331A005F12000E04750B957B1D5F810C0DCF85C
S11331B014C0042306AA414605F12000E047E8B9FB
S11331C09DF80C00C8B15EB104A80290214605A880
S11331D001904B4600F015F8324600F018F858B943
S11331E05FB104A8029006AB05A80190082200F084
S11331F008F8414600F00BF800B9002009B0BDE81A
S1133200F083A8680069006DC0B2009070472C6913
S1133210A46A05F12000204770B5044688B00D4625
S113322000204DF82020401C0828FAD375B1202630
S1133230202D98BF2E466A4631462046FFF78CFF64
S1133240002804BF3419AD1BF0D000E0002008B002
S113325070BDF8B504460D46374E384B37693F69A3
S11332602A46214606F12000B84760B9B1680969C9
S11332700A6B42B10B6D21463469646ADBB22A469B
S113328006F12000A047F2BD10B52B4C2B49226952
S1133290926804F12000904758B9A16809690A6B43
S11332A022B12269096D00F029F810B9244A0121DC
S11332B0117010BD70B5154682B000222A700A46FE
S11332C01D4C2669766C01466B4604F12000B0471C
S11332D098B99DF8001029709DF8001069B1184D37
S11332E0297851B9A06800692269016D00F006F8D7
S11332F008B16C2076BD0121297076BD126AC9B26D
S113330004F12000104710B514460B4A82B09268AD
S11333101269126B02B101224942227089088900A4
S11333206A464942FFF7C6FF20B99DF8001009B16B
S11333300021217016BD0000188FFF1F6B66656B9E
S1133340B3A7FF1F38B50446B0484068012C0CBF32
S113335000F1300500F12005FEF79CFD18B9287234
S113336040F2951032BD69461020FEF7AEF968BBF5
S1133370009820B9286868604FF4C87032BD012CE9
S113338005D1B0F1806F08D94FF0806004E0B0F14E
S1133390006F02D94FF00060009028680099091866
S11333A0491E6960012129727CB9994CA060694663
S11333B06868E0600320FEF788F900982060694699
S11333C00420FEF782F900986060002032BD70B5D9
S11333D000F07AF800B9C7E0324629462046BDE835
S11333E0704001F015B92DE9F84301280C46154643
S11333F0984603D1204600F001F90446FEF74AFD41
S11334000028834F834E08BF40F2951032D085B315
S1133410307860B93868401E044218BF40F29110F9
S113342028D1012030700020B060746002E0F068A0
S1133430A04219D1B06839682A188A423DBFA9460A
S11334402919F160A1EB000980194A464146103060
S1133450FEF7C8FFB0684844B0604C4439688842FD
S1133460C844A5EB0905D2D100F033F80028CED02A
S113347000E00020BDE8F2837CB500F025F810B927
S113348040F2951076BD012C03D1284600F0B6F821
S11334900546B408A40006F0030608E001AA0421C6
S11334A0284600F08DF80028ECD12D1D241F002C97
S11334B0F4D136B101AA3146284600F081F800283B
S11334C0E0D100F006F876BD04460D461646FEF738
S11334D0E1BC70B54F4C20780025E8B14C4EA06893
S11334E03168884205D0091A0019FF22103001F012
S11334F0C1F83268606804F11001FEF7C1F90546AD
S113350000202070A0603DB93268606804F11001A9
S113351001F0E4F800B124E0284670BD70B5FFF76F
S1133520D3FF00B920E0012C03D1284600F066F84F
S113353005463748446860420540714208404642A7
S113354001E0361B651956B12846FEF7D8FA38B99A
S11335502146284600F020F80028F2D001E000209F
S113356070BD40F2931070BD40F2951070BD80B5EF
S1133570FEF790FC10B940F2951002BDFEF77CFAFC
S113358048B923498868C968091A491C00F004F835
S113359008B140F2931002BD4942890889008008AD
S11335A04942800000E0091F31B150F8042B12F1A8
S11335B0010FF8D001207047002070470020C1E6B9
S11335C013460A46014600200DE713460A46014603
S11335D0002051E70A46014600209FE70120B1E69A
S11335E013460A4601460120FDE613460A460146F3
S11335F0012041E70A46014601208FE70349496853
S11336000A6A096B8018401A70470000188FFF1F60
S1133610E09DFF1FF09DFF1F10B504466068A16880
S1133620814211D2401A6060A1660FF2CD30206051
S1133630E08A28B104F1280104F1380001F080F88F
S11336400120A060002010BD42F2787010BD10B5BA
S113365004460021DFF8D00501F072F8616A1022F7
S113366004F12800FEF7BEFE606A00F01EF80FF2B7
S1133670050017E010B50446DFF8B035606A4289EA
S1133680A282C268921E626042689A4202D1017AA2
S1133690022902DB42F2757010BD00F006F80FF249
S11336A0150000BF2060002010BD04F13802102175
S11336B001F06BB810B5044682B0606A4268636872
S11336C0A2610268D21E9A42A26002D342F27670CC
S11336D016BD02896AB1E28204F138024189C91E29
S11336E021660FF239012160102101F04EF800200B
S11336F016BD00208DF800006946DFF8342502F17C
S113370020001269926990479DF8000010B142F2BE
S1133710817016BD2046FFF77FFF16BD10B5044625
S113372004F13802A068401EA0601021606A01F014
S11337302CF8206E401E206604BF0FF23500206076
S1133740002010BD10B5044604F12801A068401EF5
S1133750A060DFF8D40400F0F3FF606A04F13802DB
S1133760102101F03AF82046BDE8104054E700006B
S113377070B505461022A868696A461EAE6005F158
S1133780380000F0ABFF002418B9DFF8A804286063
S11337900BE0E88A401EE88280B220B1701EA86067
S11337A00120A86601E04FF41E54204670BD38B5D0
S11337B00446E08A08B100F055F8DFF874542B6829
S11337C0626A216EE06D9B689847A8B9A168206978
S11337D0491E884203D328680069804760B900F015
S11337E046F800F03AF80098616E884200D044E050
S11337F00FF205202060002032BD38B50446E08A6F
S113380008B100F02FF8DFF8285400F030F82B68E6
S1133810626AE06D9B6810219847E8B9E06D10304A
S1133820E065206E10382066112828BFDFF80804F0
S113383010D210B1DFF804040CE028680069804756
S113384050B900F00AF80098616E884200D014E084
S11338500FF2A5102060002032BD694604F11C005F
S1133860FEF7A6BB626A1021104600F0B6BF616A7B
S1133870102204F11C00FEF785BB42F27A7032BDBF
S113388010B5044604F11C00FEF776FB206E1128E7
S11338902CBFDFF8A403DFF8A40303E7DFF89033B9
S11338A01B68426E016EC06DDB681847F8B50446AC
S11338B0B4F85A00C0F30321C0074CBF08250425FF
S11338C0E66D042901D00420F2BD00F024FB04F1CC
S11338D06002DFF85C733C69646B2B46314607F188
S11338E02000A047044600F01CFB002C14BF204617
S11338F00020F2BD70B5044642F27F76E56D28469D
S113390000F0C4F980B1606E04F11801A8470646BE
S1133910012E03D12046BDE870407DE6022E03D17E
S113392000F0B3F8002070BD304670BD10B500F152
S11339305C01031D1C684A685A60944202D242F238
S1133940767010BD0A7AD2070FD50A685C69A24264
S11339500BD1496849B19960598A21B100F1280114
S1133960383000F0EDFE002010BD90F85A10C90761
S11339705CBFBDE81040FFF74FBE42F27C7010BD43
S1133980B0F85A108A070BD4CA070BD5C1F3032029
S1133990002808BFFFF778BC012808BFFFF7E7BD80
S11339A004207047A24A126852695C30416800687A
S11339B0104738B5C46DB0F85A00C0F3032001288D
S11339C004F2FF1507D1204600F060F918B128462B
S11339D000F05CF908B9042032BD2046FEF7FFF977
S11339E00400934D02D1286800688047A8680069E4
S11339F04465204632BD0000D0B5044604F15806A3
S1133A00E08A5A2708B1FFF72DFF616A3046102279
S1133A10FEF7F8FC0120815D7F18401C1028FAD3C2
S1133A203078F9B2884202D042F27970D0BD717810
S1133A300A2942F2127025D8DFE801F01A060A0EAC
S1133A4026121A16261C20002046BDE8D0406DE739
S1133A502046BDE8D04013E72046BDE8D0401DE72E
S1133A602046BDE8D04045E72046BDE8D04087E782
S1133A700020D0BD2046BDE8D0409AE72046BDE8EE
S1133A80D04013E742F27B70D0BD70B56C4C70210E
S1133A902046FEF7A3FC6B48654D206000F03BFA1E
S1133AA02E69614CB66B04232246302105F12000B7
S1133AB0B0472E69B66B0423221D312105F1200085
S1133AC0B0472E69B66B042304F10802322105F1D4
S1133AD02000B04705F120002D69AD6B042304F1EB
S1133AE00C023321A84700F01CFA002054F82010DF
S1133AF011F1010F02D1401C0428F7D3042804D18A
S1133B0000200021002200230FC4002070BDF8B55E
S1133B1004460D46002000264B4FAE4217D03869AC
S1133B20C0F11000A91B09E079B13B69325DDA5597
S1133B30761C3A69521C3A61401E491E0028F3D192
S1133B40386100F005F810B9E7E742F27D70F2BD84
S1133B503B493D4A4A620020CA682AB10B69934234
S1133B6009D0581C086101E08A6E12B90846096838
S1133B700847521E8A6670472DE9F0412C4C206894
S1133B800069804700284DD1DFF8B48098F85900C7
S1133B90042833D108F15C052E68304600F076F82D
S1133BA007000BD0FDF789FB58B1FEF776F9FDF756
S1133BB059FB00B10027FDF798FB17B940F2F71045
S1133BC030E00020FFF75EFA98F85A00800710D51D
S1133BD0686868616168103158B10A68904223BF0F
S1133BE04968491C814204201CD380F3088880F36F
S1133BF00988A868B04742F27E7013E008280FD104
S1133C000220FFF73FFABFF34F8F1048104A0168B4
S1133C1001F4E06111430160BFF34F8F00BFFDE782
S1133C2042F27B70BDE8F08188A2FF1F53544D50CF
S1133C30188FFF1F8D32FF1F4333FF1FF732FF1F03
S1133C4000A2FF1F9731FF1F74A2FF1F0CED00E0BD
S1133C500400FA0538B504460D46FEF71EF9FDF7D3
S1133C6023FB0020FFF70EFA9748984A056044604A
S1133C7000211160016881F3088881F30988406894
S1133C808047BDE832400020FFF7FCB910B582B090
S1133C9000281EBF10F1010F8D49884201D1002078
S1133CA016BD6A46022100F05BFE002418B9009894
S1133CB0007A00B10124204616BD2DE9F04FDFF84B
S1133CC01482854D83B0D8F80800006900F16807B4
S1133CD02E4609E0397C014205D07069F268816999
S1133CE0526830469047183630680028F2D10024D4
S1133CF0A146CDE900494FF47A70FEF7E7FB06468A
S1133D008A46FEF7F5FC002844D1FFF7BFFF5FEABF
S1133D10000B3FD0FDF7D1FA50B1FEF7BEF8FDF726
S1133D20A1FA00B1A346FDF7E0FABBF1000F31D0D0
S1133D30D8F80800006990F88600C00703D4002171
S1133D400020FFF787FF788A4FF6FF71884208BF8B
S1133D5041F28830A6FB00230AFB0033CDE900239F
S1133D60FEF7AAFB04468946DDE90001002908BFE5
S1133D7000280FD0FEF7A0FBDDE90023001B61EB58
S1133D800901994206D301D8904203D300210020AF
S1133D90FFF760FF2E4600E0183630680028E3D0B5
S1133DA0397C0142F8D0F168096830468847002818
S1133DB0F2D0002ED8D009E0397C014218BFAE42BF
S1133DC003D0E96889682846884718352868002898
S1133DD0F2D13046BDE8FE8F30B583B000F095F8DF
S1133DE0FEF710FC3B4C2169496804F12000884728
S1133DF0A06800688047FEF731FBFDF731FA78B31D
S1133E00A06800692369D0F89850DB6A6A460421E7
S1133E1004F1200098472369DB6A01AA012104F117
S1133E202000984715F1010F15D00098A84212D22E
S1133E3001990818A0F50070A8420CD34FF4007142
S1133E402846FDF759FA30B92846FDF7C8FF40F275
S1133E509511884202D10020FDF7C1FFFDF745FA14
S1133E6000F059F8FEF722FB00F05BF80020FEF7A3
S1133E705BFBFEF7F3FA206800688047A06840689F
S1133E808047FFF71AFFE061016919B109680A0068
S1133E9018BF8847E069416919B109680A0018BF69
S1133EA08847E0680068804737BD38B5FFF794FF5E
S1133EB0084CE569E06840688047E868C168080024
S1133EC0F8D028468847F5E7B099FF1F08ED00E0D1
S1133ED01104FF1F188FFF1F640AFF1F70470000A3
S1133EE00160704772B60168491C016062B60168DE
S1133EF00029FCD10120704772B60168491E01E017
S1133F0072B60021016062B6704772B6094900209A
S1133F10086062B6704772B606480168491C0160C1
S1133F20704704480168022900D2EAE70168491E83
S1133F3001607047E89AFF1F08B904207047DFF852
S1133F406C150968090E01F00F010F290FBF4FF41A
S1133F5080210FF2F05232F811108902002202601F
S1133F6041604FF48072012181604FF48051C1603F
S1133F70DFF83C1591F900309A404261C9788161BB
S1133F8000210161016241620020704738B50400DC
S1133F9001D1042032BDDFF81C256FF03B4000F056
S1133FA046F801D06B2032BD38E02DE9F04389B0EA
S1133FB0164680460D4600F0EAF9049B00F0E3F94A
S1133FC004001BD1009D019F7019461EB6FBF7F03B
S1133FD007FB106121B1401C7843461E00E07D19A7
S1133FE0AE4217D32802000ADFF8C81440F010606C
S1133FF00860DFF8C404814502D06B2420465BE0EE
S113400000F089F90446D8F81000010018BF804771
S1134010002CE4D0404600F03EFAEFE7204600F0E2
S113402024FA0546204600F036FA284632BD1060D0
S1134030DFF88404814270472DE9F04389B00446D7
S11340405FEA02080F461D4608BF042034D000F082
S11340509FF9039B2A463946204600F03FFA5FEA5F
S1134060000929D1009FDFF84C6402E00398C719C6
S11340702D1AEDB158F8040B706039020398090A3F
S1134080042808BF41F0C06006D0082805D158F8BC
S1134090040BB06041F0E0603060204600F0E5F9C8
S11340A081462069010018BF8047B9F1000FDDD0B7
S11340B0204600F0F0F9484609B0BDE8F08370B539
S11340C0040018BF002A01D1042070BDDFF8E40306
S11340D0DFF8E863CDB246EA0545056010291568A6
S11340E0456002D01139032903D2082B04BF51685B
S11340F08160204600F0B9F90546204600F0CBF96E
S1134100284670BD2DE9F04389B05FEA0008914666
S113411014BFB9F1000F04200E461D4647D000F02D
S113412037F90698401E064208BF05421AD1A9195C
S1134130109C0020491E012C05D1002E04BF691ECD
S113414007290AD10AE044B9FF2907D9B6F5000FB7
S113415003D3DFF86C23914200D3042038BBDFF88B
S113416054730DE0652022E0796849F8041B069930
S1134170082904BFB96849F8041B06998E196D1AF9
S1134180ADB13002000A40F0407038602006069954
S113419040F0FF1040F47F40042908BFB86002D00B
S11341A0082908BF786000F0B6F80028DCD083E75F
S11341B0F8B51546002818BF002D0C461E4601D13F
S11341C00420F2BDDFF8EC72DFF8F822E1B242EA33
S11341D00141396000F049F958B979682960102C17
S11341E003D0A4F11101032903D2082E04BFB96836
S11341F06960F2BD002818BF002901D1042070476E
S1134200DFF8C402007800F00302022A08BF00208D
S113421005D000F0C00080280CBF012002200870E7
S11342200020704710B50A46002818BF002A01D1A3
S1134230042010BDDFF890321C78002104F0030440
S1134240022C1ED06FF03A41C3F802105478117852
S1134250240444EA0161947841EA0421D478214396
S1134260C3F8061054791179240444EA016194795D
S1134270D27941EA04211143C3F80A1000F0F5F899
S11342800146084610BD08B904207047DFF83C22F7
S113429080E02DE9F04F89B0924680460C4600F04C
S11342A076F8059B52462146404600F017F978BB44
S11342B06A462146404600F026F9009C029E604270
S11342C0714208404542A54208BF7519794F03E081
S11342D0AAEB0B0A5C447519BAF1000F17D0281B1E
S11342E0D346824588BF83460598BBFBF0F0210284
S11342F0090A000441F0807140EA0920396040F065
S1134300FF00786000F007F80028E1D000E000200A
S113431009B0BDE8F08F4046A7E02DE9F04389B02D
S113432080465FEA03090D46164608BF042029D0DB
S113433000F02EF8079B00F026F818BB009D109C97
S11343405C4F05E007998A08761A09EB82094D1932
S1134350C6B12802000A40F000703860200640F020
S1134360FF1040F47F407860D9F80000B860FFF790
S1134370D2FF0028E6D0119901B10D60129909B15C
S113438000220A6098E6324629464046A6E099464D
S11343906A46B8E042EA0141464A116065E02DE907
S11343A0F04180461E000D46174608BF042034D055
S11343B0042300F093F880BBD8F814307A195F42D4
S11343C0C2F1000C07EA0C0CCCF1000C2F40ACEB52
S11343D007070021B7FBF3F7DFF8F4C00AE0DCF8C5
S11343E000E0203C6FEA0E0E2EFA04F4E40748BF06
S11343F0491C5D1995420AD2B5FBF3F4202C38BF51
S1134400DCF804E0EED3D8F818E07445E7D319B12A
S1134410B94234BF022101213170BDE8F0810000AE
S1134420002818BF002A01D10420704709291AD88E
S1134430DFE801F00509090B0D0F11131517C0680A
S11344401060002070474068FAE78068F8E7006869
S1134450F6E70120F4E74069F2E78069F0E7006AD3
S1134460EEE7406AECE76A2070471A487021017051
S11344708021017001780906FCD50078810601D5F8
S113448067207047C10601D568207047C0074CBF3C
S11344906920002070471049096851F470010E4AE0
S11344A01160BFF36F8FBFF34F8F70474C80044090
S11344B028000240040002406B66656BFFFF004366
S11344C000048000FFFF004102000240FFFF0040A3
S11344D0180002400000024004F0014008B9042022
S11344E070475B1E194208BF1A4201D0652070470D
S11344F00368994221BF4068C0185118884234BFEC
S113450066200020704770B505000E46144601D1A0
S1134510042070BD20212046FDF760FF2868301A72
S11345202060E8686060A9686868B0FBF1F0A0608A
S11345300420E0601020206160610420A061E0613B
S1134540002070BD0800100018002000300040005A
S113455060008000C000000180010002000300042C
S11345600006000080B51B491B4808601B491C4815
S1134570421A1C4888421CBF002AFDF733FF1A4820
S11345801A49091A18BF00F03BFA19481949091ABF
S113459018BF00F035FA18491848421A04D0BDE88B
S11345A008401748FDF71EBF01BD16484FF0FF3104
S11345B0016041608160C160016141618161C161EB
S11345C01148016041608160C160016141618161A4
S11345D0C161704708ED00E00000FF1FBC8AFF1FA7
S11345E0308EFF1F088FFF1F2099FF1FB4A7FF1FE6
S11345F00094FF1F2099FF1F088FFF1F088FFF1FC4
S1134600B4A7FF1F80E100E080E200E000F0FCB905
S1134610134680B50A4601461846FDF7E3FE00201E
S113462002BD70B510F0030F0C46154612D0B0F160
S1134630005F0FD22118491EB1F1005F0AD3C0F107
S1134640005632462946FDF7CDFEA21B71194FF0E4
S1134650005001E022462946FDF7C4FE002070BD4B
S113466010B514460A462146BDE810400123FCF764
S11346705BB9000062F30F2262F31F42401810F08E
S1134680030308D0C91A1FD3DB0748BF00F8012D64
S113469028BF20F8022D130030B4144615461039F3
S11346A028BF20E93C00FAD8490728BF20E90C00BC
S11346B048BF40F8042D890028BF20F8022D48BFC8
S11346C000F8012D30BC7047C91818BF00F8012D3F
S11346D0CB0728BF00F8012D70470000030000201D
S11346E013F0030F09D0521E22BF13F8010B11F867
S11346F001CBB0EB0C00F3D07047121F22BF53F86C
S1134700040B51F804CB6045F7D0121D0AD200BA4D
S11347109CFA8CFCB0EB0C0038BF6FF0000088BF33
S113472001207047521E22BF13F8010B11F801CB70
S1134730B0EB0C00F6D0521C08BF104670470000C6
S113474070B50D46424C30B10146102204F1100000
S1134750FDF748FE06E004F11000002100220023CA
S113476000264EC02DB1102229462046FDF73AFE00
S113477005E000200021002200230FC4103C04F1B6
S11347801000BDE87040FCF742BD2DE9FF4100F088
S113479058F81EE000F050F8009831684840009046
S11347A06A46019871684840019010340298B168D3
S11347B0484002907F1C0398F1684840039006F13A
S11347C010016846FCF72EFD684600F043F8103EE1
S11347D010354745DED3BDE8FF812DE9F04188B0AF
S11347E000F02FF823E01022214604A8FDF7FAFD7B
S11347F000F022F86A4606F110016846FCF71EFD37
S1134800009831684840009010340198716848401D
S113481001907F1C0298B16848400290F1680398A7
S11348204840039004A800F015F8103E10354745A1
S1134830D9D308B0BDE8F081102221466846FDF7BF
S1134840D1BD044615464FEA11180027004E7047A3
S1134850B899FF1FB0E80E10A6E80E1010226946A2
S11348602846FDF7BFBD000070B50D0082B00446B8
S1134870164601D1002076BD6A4600F071F830B9C1
S1134880009BDB685B68324629462046984776BD24
S113489070B50D0082B00446164601D1002076BDE5
S11348A000F07FF800B14CE000F047F868B9009BD5
S11348B0DB689B6832462946204698474E490028C3
S11348C006BF009AD26800220A6076BD38B5044655
S11348D00D466A4600F044F8A0B90098C0684069E3
S11348E008B9662032BD2946204600F05AF810B1B6
S11348F042F2D87032BD009AD268526929462046E5
S1134900904732BD002DFCD1002032BD70B50D00A2
S113491082B00446164601D1002076BD00F041F86D
S113492000B10EE000F009F830B9009BDB68DB68E9
S1134930324629462046984776BD6A46294620468F
S11349400EE042F2D87076BD10B52B4C21680020E1
S113495029B109690A0002D088470021216010BDED
S113496070B542F2D873D2B1244C6468146011B9A2
S113497015E01034146014688CB12568002D04BF50
S11349806668002E01D1E6684EB1A84224BF65686E
S11349908542EED30818401E854228BF00231846DE
S11349A070BD70B50918491E0022144B9C685D68DF
S11349B02469160104EBC2045834755966682468E6
S11349C0AC4208BFAE4205D0864228BFA14201D303
S11349D0012070BD521C022AE8D3002070BD10B51E
S11349E00648446804E00068010018BF804710349A
S11349F0E0680028F7D110BDFC9AFF1F188FFF1F35
S1134A000022FFF73BBE00001D480068000B00F0C9
S1134A100F00C01E082830D8DFE800F005080B0E90
S1134A201114172F1A004FF4804013E04FF4C040C4
S1134A3010E04FF400400DE04FF440400AE04FF422
S1134A40803007E04FF4C03004E04FF4003001E060
S1134A504FF480200321421E10420A4A18BF02214B
S1134A6052684B1CB0FBF3F0C0F1005342F8103F06
S1134A706FF0604301FB003050600020704700BFBE
S1134A8000700440188FFF1F02280ED80FF2240272
S1134A9080560122012900F01F0102FA01F10CBF26
S1134AA0024A034A400942F82010704700E100E03E
S1134AB080E100E01A1B4100BFF34F8F0548064A0E
S1134AC0016801F4E06111430160BFF34F8F00BF3F
S1134AD0FDE700000CED00E00400FA05ECE7EBE76D
S1134AE0EAE7E9E702280ED80FF2240280560122F1
S1134AF0012900F01F0102FA01F10CBF024A034A26
S1134B00400942F82010704700E100E080E100E035
S1134B1018194A0004280ED80FF2240280560122E4
S1134B20012900F01F0102FA01F10CBF024A034AF5
S1134B30400942F82010704700E100E080E100E005
S1134B401E1F20212200000040684A49405C704733
S1134B504849CA6842B18A6813780370501C886057
S1134B60C868401EC86070470021017070475A2809
S1134B7007D1404A01238B540FF209015161916915
S1134B80084770473B49896908477FB5394DA96192
S1134B9004460FF2FC00616850F82160684600F09A
S1134BA0F7F801208DF808008DF809000221324839
S1134BB0286132486861A268606890476946304657
S1134BC000F097F82E49304600F014F9606801218E
S1134BD0FFF75AFF616849190120087104B00020E9
S1134BE070BD70B50546234C68680119097989B10F
S1134BF00FF29C0151F820600021FFF745FF304679
S1134C0000F0D2F86868AA68002190476968091919
S1134C100020087170BD17488160C260C168002916
S1134C20FCD10020704770B504460FF2640082B0D6
S1134C3050F82450E86A00010BD54FF0006007E0FB
S1134C403169684688479DF8000068634FF000703A
S1134C50E862E86A074E8001F2D4E86A800308D566
S1134C60A86B4FF40031E96221467269C0B29047E3
S1134C70F3E773BD948FFF1F9946FF1FB746FF1FCD
S1134C800000020A0020CEE70120CCE70220CAE798
S1134C9000C0024000D0024000C00A40010C01F1F3
S1134CA0804101F58E2101230A6803FA00F01043C4
S1134CB0086070470029016814BF21F4804141F461
S1134CC080410160704700210FF2140252F8213034
S1134CD0834202D0491C0329F8D3084670470000D8
S1134CE000C0024000D0024000C00A40012120461A
S1134CF0E0E738B504460D46FFF7E5FF00F043F85A
S1134D00FFF7F4FF00F088F8012220684000400813
S1134D10206020680840297B40EA8170A97B40EA32
S1134D208160697B40EA0160E97B00F019F80121A8
S1134D30204600F054F8287804EB8000C1686A68C3
S1134D4000F014F82A7A920602F0806211436A7A1B
S1134D50520602F000721143C16000F00FF831BD39
S1134D60090201F44071084320607047521ED206C4
S1134D7021F0FE4102F0F0421143704720684008E0
S1134D804000206070470FF2A00151F8200085E731
S1134D9000210170082141600021017241720173F8
S1134DA041738173C173704710B5044600212068B4
S1134DB000F034F8FFF79BFF00F02CF80FF26801C5
S1134DC051F82000010C01F1804101F58E210123ED
S1134DD00A6803FA00F022EA0000086010BD0368C4
S1134DE0090401F47C11012A0CBF194323EA0101CF
S1134DF0016070478A0103D5026B22F0807202635E
S1134E008A0303D5026B22F480320263026B1143DE
S1134E1001637047204656E72068024940F00100CC
S1134E2020607047FFCCFFBA0C003C100D003C1012
S1134E300C003010010C01F1804101F58E21012399
S1134E400A6803FA00F0104308607047010C01F18E
S1134E50804101F58E2101230A6803FA00F022EA59
S1134E600000086070470029817814BF41F0800178
S1134E7001F07F018170704700210FF2F00252F8B7
S1134E802130834202D0491C0429F8D308467047D4
S1134E904A0603D5827842F040028270890603D51F
S1134EA0817941F0200181717047C178827952067D
S1134EB048BF41F480418079C00648BF41F4805125
S1134EC00846704738B504460D46FFF7D5FF00F095
S1134ED030F8A87A10B1022804D00DE0E888400028
S1134EE0207009E0E8884000207028894000E071C3
S1134EF0607940F008006071A078A97800F0FD00A6
S1134F0040EA4100297840EAC110A070607929790B
S1134F1000F06F0040EA0110697840EAC110E978B6
S1134F2000F001F831BD00F0DF0040EA411060718B
S1134F3070470FF2480151F820007BE710B5044692
S1134F400021FFF790FF2046FFF796FF0FF22C0198
S1134F5051F82000BDE8104078E7002181724170CB
S1134F608170C170017101210170704700600640B9
S1134F700070064000600E4000700E4006003410C1
S1134F8007003410060028100700281000210FF233
S1134F90C81252F82130834202D0491C0529F8D3A3
S1134FA0084670472DE9F0410D460446286800265E
S1134FB00146B046042303FB00FCB2FBFCFC1FFAD1
S1134FC08CFCBCF1000F08BF4FF0010C0CF1010781
S1134FD00CFB03FE5F43B2FBFEFEB2FBF7F7AEEB46
S1134FE0000EC71B77453CBFBE460CF1010C714552
S1134FF002D371461E46E0465B1C212BDBD36422A0
S1135000B0FBF2F000EB4000884238BF40F2215080
S11350104ED32046FFF7BAFF00F05EF81043086055
S1135020311FA06820F44020A06004292068DFF824
S1135030241138BF40F400300840711E090601F005
S1135040F85108434FEAC84150EAD1402060206833
S113505020F000502060A06820F01000A060A0683C
S113506080088000A060A06829790843A0602068B7
S11350706979490320F4005001F400510843206089
S1135080A979E87941EA0040E061A06940F088002C
S1135090A061A06940F44040A061A068297A09B1E8
S11350A040F40020697A09B140F48020A060002017
S11350B0BDE8F08180B5C16911F47F4FFBD141682F
S11350C04902FCD500218160FFF760FF00F004F87D
S11350D022EA0000086001BD0FF2900151F820009F
S11350E0010C01F1804101F58E2101230A6803FAC4
S11350F000F070474FF4E13101600021017141710A
S11351008171C17101724172704710B50A0203685E
S113511002F440442343036002F4407283691A4357
S11351208261090A826842EA0121816010BD4168F6
S11351308069000C00F0C3000843704705E0436831
S11351401B02FCD511F8013BC36013465A1E002B09
S1135150F5D1704700E0FFE000400C4000500C40E7
S113516000600C4000700C4000600D4004002C10E6
S113517005002C1006002C1007002C1016002C1013
S113518070B5424E01243068491E1546082900F1C5
S11351900C024CD8DFE801F0051423424228424BAC
S11351A04000696811F1010F18BF00290ED0D168C1
S11351B0012912DB90F8461001290ED118300AE0BB
S11351C0696811F1010F18BF002901D1002070BDD9
S11351D0116114701430FEF78FFE002427E024219F
S11351E02030FDF7FBF822E0A978002904BFE97814
S11351F0002904D12978012908BF547017D06A689E
S113520029462030FDF7EEF830686968C1610473FF
S11352101430FEF771FE0AE0052408E00021143082
S1135220FEF75EFE306800211830FEF759FE204676
S113523070BD38B50C460020012C0DD1134D2868E3
S113524080F8461000F1200280682423022100F037
S1135250C8F9296881F8474032BD002051B90B488C
S1135260006880F8482000F120028068242302218D
S113527000F0B7B97047054908600020704703493A
S1135280086000200968886070470000EC9AFF1FDE
S113529010B5134601200BB9032010BD00225A7427
S11352A05A6832B11468220003D00A460121184614
S11352B0A04710BD10B5134601200BB9032010BD43
S11352C000229A745A6832B11468220003D00A4644
S11352D002211846A04710BD2DE9FF4104460025D0
S11352E061688968227B4B79012093424ED3096817
S11352F000294BD001EBC2010839002200E0521C06
S11353000B789A4242DA4B680C2606FB02331E786D
S1135310032EF4D194F80EC0002100E0491C1A7A3F
S1135320914205DA5A680E01B75C6745F6D1B518A3
S1135330D978617355B3A5604FF00008974E984F24
S113534007E0039402AA2068694600F059FA08F1BC
S113535001082979884519DA00208DF80400A86825
S113536010F828008DF80200C009A96801EB880133
S113537001284988ADF80010A96801EB8801497833
S11353808DF803100CBF02970296DAE704B0BDE86B
S1135390F08138B504460120A16861B1002506E01A
S11353A0886810F82510206800F047FA6D1CA16881
S11353B00A799542F4DB32BD70B5044615460120E6
S11353C084B0002D14BF002C03200BD0491E0529E6
S11353D008D8DFE801F05A0308182E44002121738D
S11353E06174A174B9E0616800291EBF217B2A7829
S11353F08A42F7D011B12046FFF7CBFF28782073FB
S11354000020A07311E061680029EBD02988627B39
S11354100D460904B2EB116F0AD1A17BEDB28D42A6
S113542006D02046FFF7B5FFA5732046FFF754FFCB
S113543093E0616800291CBFA1680029F8D0002608
S1135440A26811798E42F3DA9268297812F826203C
S1135450914204BF206800F008FA761CF0E7616806
S113546000291CBFA168002977D00026A268117901
S11354708E4272DA9268297812F82620914204BF8B
S1135480206800F0FCF9761CF0E729680A7802F03D
S11354901F02012A02BF0A79637B9A425DD14A78CE
S11354A0012A20460AD0022A13D0032A1AD0092A34
S11354B022D00A2A40D00B2A45D04DE04988090A57
S11354C08DF808106A46296849888DF80910032167
S11354D020E063681B6804F10F020421984704F17B
S11354E00F0107E063681B6804F110020421984768
S11354F004F11001696030E04988090A8DF8081048
S1135500296849888DF80910297B59B1A968019146
S11355106A46092163681B68984700996960019984
S1135520A9601AE0696800916A46A9680191062198
S113553063681B68984710E04988090AE173296881
S11355408A1C072104E04988217404F1100208210F
S113555063681B68984700E0052004B070BD70B50F
S11355600C461546002114230E4A03FB012632681B
S113557022B1491C0129F7DB022070BD314600F03D
S11355801CFA50B9306808B9032070BD002030738C
S11355907460FF20B0732E60002070BDFD4DFF1FAE
S11355A0D94DFF1FA496FF1F10B5040001D103209D
S11355B010BDFFF7EEFE0021216061602173A1732D
S11355C010BD10B5040001D1032010BD607C08B1EA
S11355D0022010BD206800F001F908B901216174AE
S11355E010BD10B5040001D1032010BDA07C08B18A
S11355F0022010BD206800F0F6F808B90121A1745A
S113560010BD000010B5044600F0DCFA0020206054
S113561084F88D0000F0E0FA002010BD38B508B918
S1135620032032BD446844B100680D0602D5A46865
S1135630A04732BDE468A04732BD062032BD08B998
S113564003207047436813B100685B69184706205C
S113565070473EB504460A7AD5090120102A02F0A3
S11356600F0319D100220B212046FFF7E8FF04F1B4
S11356708C0002218170002200210170002004EBC3
S1135680C001401C1028CA600A61F8D3A368012134
S11356902046984700203EBD082B11D245EA43021C
S11356A004EBC203DA685AB10868009048680190B4
S11356B0487A8DF8080069461A69DB6820469847DD
S11356C03EBD002918BF002801D10320704782681D
S11356D0002A18BFFFF7BDBF012070472DE9F04134
S11356E007461400884608BF032053D000F06AFA26
S11356F0294D286805F18C0630B171788F4203D1A9
S113570000F06AFA01273FE018B100F065FA0227B9
S11357103AE0777000F060FA0020C5F808807770EE
S11357203070002205EBC001401C1028CA600A61D9
S1135730F8D3012F19D80FF2F81068601748002821
S11357401CBF174800280BD0164800281CBF164859
S1135750002805D0154800281CBF1548002809D189
S11357602846FFF74FFF072014E02846FFF74AFFBB
S113577006200FE02A462946384600F05AFC070066
S113578004D0284600F019F8384603E00220B0702F
S113579025600020BDE8F0811496FF1F7B5BFF1F8E
S11357A0E95BFF1F235CFF1F915CFF1F375DFF1F39
S11357B0795DFF1F0022002141E710B5040001D1EB
S11357C0032010BD616821B1206849688847002022
S11357D060602046FFF716FF002010BD01F00F01A6
S11357E041F080011AE701F00F0117E708B903201F
S11357F07047426812B1006812691047062070476A
S113580010B508B9032010BD002918BF002A12D012
S11358108B7803F00F04082C0DD2640044EAD313F0
S113582000EBC3031468DC6052681A610A46BDE8E1
S11358301040022103E7042010BD73B5044601F0B3
S11358400F05CE090CB9032076BD01AA0321FFF789
S1135850F6FE082D07D246EA450104EBC1010022F9
S1135860CA600A6176BD042076BD02B501F00F015D
S1135870082902D26A4604210BE0042002BD02B5C5
S113588001F00F01082902D26A46052101E0042033
S113589002BDFFF7D4FE02BD0000000010B50123D5
S11358A00AB9042010BD891E062900F18C0417D8FA
S11358B0DFE801F004060E10080A12000C210CE0C7
S11358C00D210AE0A07800E020780023107007E0A2
S11358D0062102E0072100E00921FFF7B0FE03469C
S11358E0184610BD10B50123032900F18C0406D01D
S11358F0062906D0072908D0092913D016E00E215D
S113590011E09AB11078002307E0A178032906D0AA
S113591062B11078207000230320A07006E02246B4
S1135920082100E00A21FFF78AFE0346184610BD4D
S11359307B5BFF1FE95BFF1F235CFF1F915CFF1F65
S1135940375DFF1F795DFF1F10B5044600F03AF97B
S113595000F027F851B1817C8C4207D1002101600D
S11359604160817400F038F9002010BD00F034F972
S1135970042010BD38B500F017F800F012F819B182
S1135980817C8C4200D113E007E038B500F00CF8BC
S113599000F007F88C4200D10AE000F01DF9042061
S11359A032BD61480168704704460D4600F00AB9EB
S11359B0286000F011F9002032BD38B5FFF7F4FF7C
S11359C0FFF7EFFF21B1807C844201D12960F0E729
S11359D0E3E7F8B50C46154601261DB16946FFF705
S11359E0D4FF08B10420F2BD002705E0491CC9B268
S11359F0032907D37F1CFFB200984068017A8F42C5
S1135A001CDA002102680C2313FB07230FF2841213
S1135A10D3F808E09EF804E002EB011C9CF80C208B
S1135A207245E3D15868DCF808302A462146984785
S1135A30052804D00028DDD10026DBE73046F2BD7E
S1135A4070B582B00D46044616466946FFF79DFFC1
S1135A5088B9012D08D10099204600F06CFF009A06
S1135A6002212046FFF7B5FF009B5B685B68324666
S1135A7029462046984776BD2DE9F84391460124EE
S1135A800F46B9F1000F18BF002F804601D0786887
S1135A9008B9042045E000F095F8234E306828B199
S1135AA0B17C884502D100F097F816E018B100F0F7
S1135AB093F8022411E086F8128000F08DF87760E4
S1135AC032461A494046FFF709FE040007D0306801
S1135AD0FFF773FE4046FFF737FF204621E000271B
S1135AE00FF2B00415E00025706800680C2111FB6A
S1135AF007012B01886800791A19127B904203D19F
S1135B001B590A1D404698476D1C032DECD37F1C7E
S1135B10FFB27068007A8742E5DB3068C9F800009C
S1135B200020BDE8F28300000096FF1F8955FF1F87
S1135B3070B582B004466946FFF71CFF050027D103
S1135B40002517E000260098406800680C2111FB2E
S1135B5005000FF240018268127901EB06110B7BFC
S1135B609A4202D1406849688847761C032EEAD3DA
S1135B706D1CEDB200984068007A8542E2DB009823
S1135B800068FFF71AFE050004BF2046FFF7DCFE9D
S1135B90284676BDA750FF1FF150FF1F014FFF1F7E
S1135BA001000000E97CFF1FDD7DFF1FF97DFF1F61
S1135BB003000000000000000000000000000000DE
S1135BC0000000000A480178002900D172B601786B
S1135BD0491C0170704700000548017800291FBF67
S1135BE0491E0170C9B2002900D162B67047000095
S1135BF01C99FF1F2DE9F04104461D460E46174629
S1135C00FFF7E0FF47EA460804EB081006F00F022E
S1135C10C16A41F48043C36207F001016668760AF1
S1135C20760246EA42165B0A46EA011603F00803C6
S1135C3033435D606368C06A5B0A5B0243EA4212F5
S1135C4042EA0111420A02F008021143069A92053F
S1135C504009920D00F0400040EA024040F0880004
S1135C600860FFF7B9FF00F00CF9BDE8F08180B5DA
S1135C70C16A4A0A02F0080212180C32026221F4C4
S1135C8000610022826241F4005108224262C16232
S1135C9000920022036A0021FFF7ACFF01BD70B53A
S1135CA0011DFF224B6883F888204B6893F89440C9
S1135CB044F0020483F8944000234C6884F898303C
S1135CC00E68760A03F00F04760246EA44160025AD
S1135CD000F038F846F0080600F034F846F01006F4
S1135CE035600E68760A760246EA441444F01804D5
S1135CF0256000EB43150024EC6200255C0044F0B1
S1135D00010400EB0414E5624C6804EB83045B1C9F
S1135D10082B84F8C050D3D300F5907005704B68FD
S1135D2093F8944004F0FD0483F894404B6883F89E
S1135D308C2089224B6883F884204570486800F0E1
S1135D4008F870BD35600E68760A760246EA441695
S1135D50704790F8941001F0DF0180F894107047B8
S1135D6070B50C888B78C97803F00F02DB09012920
S1135D7043EA420505D1B4F5806F0ED340F2FF34F7
S1135D800BE0412C28BF4024816801EB820191F88B
S1135D90C06046F0010681F8C06000EB0511002BDD
S1135DA0CD6A25F48045CD6264F30905CD62CC6AE1
S1135DB024F40064CC6224F48064CC6214BF042113
S1135DC00821846804EB820494F8C050294384F8C1
S1135DD0C01053EA020108BFFFF749FF002070BD5D
S1135DE070B5044601F00F05C80940EA450620468F
S1135DF000F0FDF9A06800EB8500002180F8C010D8
S1135E0004EB0610C16A890A8902C162002070BDD0
S1135E1070B5044601F00F00C90941EA400204EBE1
S1135E200212D36A23F48063D36223F40063D3623F
S1135E3000236668450145EA0115760A45EA4625C8
S1135E4003F0010645EAC6052E68760705D5D66A2D
S1135E50B605B60946F008062E605B1C022BE8D393
S1135E60A26802EB8002084392F8C03003F0FD03FD
S1135E7082F8C03004BF2046FFF7F9FE00F001F8B5
S1135E8070BDA06890F8941001F0DF0180F89410C0
S1135E90002070472DE9F047044684B0A06808222A
S1135EA08030017C0270C1F303186068400A40022C
S1135EB0C1F3C00A40EA4810C1F3800140EA0A1065
S1135EC040EAC1000068C0F30949C0F383000D280B
S1135ED04AEA480004EB00150CBF01270027E86AD2
S1135EE0C0F3803000284FD004F5907007B1C17022
S1135EF0BAF1000F35D0A96A4944A9626A6A561AF0
S1135F00E96A81F40061E96281F48051E96203D0B5
S1135F108905B9EB915F1CD2A96A0191296A0091A4
S1135F20E96A21F48041E9628905B9EB915F08BF10
S1135F30B8F1000F1BD1C078696A04EBC000408A35
S1135F40814214D22068002300220021FFF746FC7E
S1135F501AE02A6A334648F08001204600F0BDF872
S1135F6012E059EA080111D100200190009048EA9A
S1135F70CA108DF808008DF8097069462068FFF78B
S1135F80A0FBA068FFF7E5FEBDE8FF87E96AC1F35F
S1135F904033BBB963685B0A5B02490A43EA4812AF
S1135FA001F00801114349682A6AAB6A9A189142C0
S1135FB006D0002302E05E5C9E545B1C4B45FAD382
S1135FC000210170A86A4844A862696A0E1AB8F1EF
S1135FD0000F0DD167B18021204600F008F9E06A76
S1135FE040F40060E062E06B40F40060E06303E0D2
S1135FF0E86A80F40060E862E86A80F48050E8624D
S1136000696A002918BF002E03D08005B9EB905FA0
S113601008D2A86A0190286A0090E86A20F48040B7
S1136020E862A4E72A6A33464146204600F08CF829
S1136030AAE770B515460FF2CC3282B0136800930C
S11360400C4630BB144E86F8220106F59271009876
S1136050F161B060FF2180F88010002201213046F8
S113606000F0E6F80D48B1687060000A81F89C0001
S1136070B1687068000C81F8B000B1687068000EF7
S113608081F8B4003046FFF70AFE2E603460002029
S113609076BD062076BD0000B896FF1F0094FF1F52
S11360A008B9032070478268FF2182F88010816854
S11360B091F88420002281F884200021826882F8EB
S11360C09810826882F89410806890F8001141F06A
S11360D0C00180F80011002070472DE9F04180468E
S11360E001F00F00400040F0010008EB001782B0FF
S11360F0F86A1D460126C0F3803030B9B8623A62AE
S11361007D62F86A40F40050F86201F00F04F86A06
S11361108005800DA84238BF054698F8210148B98A
S11361200095386AB96A0B18012221464046FFF7E8
S113613061FD0646B86A284302BF002C4046FFF7BB
S113614096FD3046BDE8F6812DE9F041044601F0A4
S11361500F00400004EB001782B0F86A1E460125C8
S1136160C0F3803010B9B8623A627E62F86A40F4D3
S1136170005083059B0DF862B34238BF1E46BB6ACC
S1136180D4F81CC09B18BCF1000F04F5907211D018
S113619092F800C0BCF1000F0CD1412E0AD216F0C7
S11361A0030F08BF13F0030C04D020F40050F8626E
S11361B0E369157001F00F08507830B90096002299
S11361C041462046FFF716FD0546002E08BFB8F1EC
S11361D0000F09D1F86A80F48050F86220F48040FE
S11361E0F8622046FFF743FD2846BDE8F681E0B596
S11361F001F00F03CA0942EA430200EB0212D36A18
S1136200C3F380338BB14FF0FF330193136A8DF8DE
S11362100810009300218DF80910D16A21F48041FF
S1136220D16269460068FFF74CFA00200EBD0000F9
S1136230F8B504460B46114601200CB90320F2BD03
S11362400C2BFCD8DFE803F0072030363D676D7077
S1136250819D9D879A00A168002081F80001A068B3
S1136260017F490703D5017F41F080010177A068D0
S113627090F8081141F0100180F80811A06890F816
S1136280941041F0010143E0A068017F490703D560
S1136290017F01F07F010177A06890F8081101F0F7
S11362A0EF0180F8081167E000296AD02046BDE8B4
S11362B0F44055E5002964D02046BDE8F44009784F
S11362C08EE500295DD00A781146204602F00F05BC
S11362D0D609FFF78CFF46EA450704EB0710C16AAD
S11362E041F48061C1624A0A6068400A400240EA9F
S11362F0451040EA061002F0080289051043890996
S113630041F08C010160A06890F8941001F0DF0165
S113631080F8941030E0A1B32046BDE8F440097839
S113632076E571B3088027E059B30A7802F00F03C9
S1136330082B26D2D00940EA430004EB0010C06ABF
S1136340800A00F00100488016E0D1B10878A16805
S113635081F8980010E0002545F08001C9B220467C
S1136360FFF73EFDE9B22046FFF73AFD6D1C082D0C
S1136370F2D32046FFF793FC0020F2BD09B10020C0
S11363800870F2BD00B970473EB50468A06890F883
S11363908050280744BF2046FFF77CFDE80712D54C
S11363A0A168012084F8210181F880006946002059
S11363B0009010208DF80800002001908DF809004D
S11363C02068FFF77EF9280615D5A168802081F89A
S11363D08000E06BC0F38020002802BFE06AC0F3B5
S11363E08020002807D080212046FFF711FD0021DE
S11363F02046FFF70DFDA06890F85C1109B180F804
S11364005C1137BD002007402DE9FC4104460F46CE
S1136410904620681E4601AA0621FFF73FFA9DF820
S113642004000525012818BF00282ED138781F2123
S1136430084208D1206804F110020421FFF72EFA63
S11364400546207C18E000F01F01012902D1002537
S1136450258214E000F01F00022812D1B8888DF8BC
S113646000006A460020ADF8020005212068FFF70D
S113647015FA05469DF8020000F003002082022070
S1136480306004F11000C8F800002846BDE8F68129
S113649070B582B0054600208DF800000C462868CF
S11364A00DF101020621FFF7F9F99DF80100052617
S11364B0012818BF002801D0052076BD6078032884
S11364C004BF01208DF8000020781F21084208D164
S11364D0608801282BD128686A461021FFF7B0FA9A
S11364E024E000F01F00022804BF608800281ED1A9
S11364F0A0880F2108420ED100F00F019DF8002062
S113650041EAD0112868002AC9B202D0FFF7ADF9D8
S113651001E0FFF7B4F99DF800102868002919BFBD
S1136520221D0521221D0621FFF753FA0646304697
S113653076BD38B500F0B6F89DF8000003280BD0FE
S1136540012818BF022801D0052032BD68888DF8C3
S113655000006A4607210AE0206800220721FFF7AD
S1136560C1F938B901208DF800006A460621206877
S1136570FFF7B8F932BD2DE9FF470646904630686B
S11365800C469A4603AA06216788FFF787F99DF807
S11365900C003D0A01284FF0050903D0010018BF83
S11365A002283AD1E0880190012D02D16A460921DE
S11365B029E0022D04D18DF808706A460A2122E0F0
S11365C0032D07D18DF80A706A46A088ADF808003B
S11365D00B2118E0212D05D1A0888DF808006A460A
S11365E00C2110E0222D05D1A0888DF808006A4600
S11365F00D2108E0232D0AD18DF808706A46A08881
S11366008DF809000E213068FFF71AFA81460098C8
S1136610C8F800000198CAF80000484604B0BDE874
S1136620F08770B5044682B0154620681E466A4657
S11366300621FFF733F99DF80000012818BF002850
S113664001D0052076BD0120306004F1100204F170
S11366501000286011212068FFF7F2F976BD38B5E3
S113666000F020F89DF80000012818BF002801D090
S1136670052032BD002000F00EF8688810B9012012
S113668000F009F82068AA1C0321FFF7A2F920688A
S1136690AA1C07213AE08DF800006A46206806210A
S11366A0FFF720B904460D4620686A460621FFF725
S11366B0F5B8F8B500F043F89DF8000008B10520DE
S11366C0F2BD0120386004F1100204F110003060C2
S11366D01221287920822068FFF7B2F9F2BD38B57B
S11366E0FFF7E0FF9DF8000008B1052032BDA8883F
S11366F0A97841EA0020208204F1100220680421D4
S1136700FFF767F9206804F110020821FFF798F9F0
S113671032BDF8B500F013F89DF8000008B105206B
S1136720F2BDA888208204F1100220680821FFF736
S1136730B5F804F11001316002213960F2BD04465C
S11367400D46164620681F466A460621FFF7A6B87E
S113675038B504460120052A0D460FD12978602258
S1136760114205D0090603D4E98809B103B9002010
S1136770C1012046BDE83440FFF777B80598E988A1
S11367800268914238BF01600368049802680021DE
S11367902046FFF723F858B92978090608D520467A
S11367A001B0BDE83040002300220021FFF71BB8F0
S11367B032BD2DE9F0418AB0044600200D46039015
S11367C0049005276868904610F1010F18BFB8F1CE
S11367D0000F10D002AA06212046FFF75FF8287A9E
S11367E00FF2B01C002808F1080649D06868082890
S11367F001D1286808B9052076E0418871806025B8
S11368008188B180C188F1804278727003783370D6
S11368102B420AD15CF8225028002DD004AB03AAE5
S113682031464046A847074626E0B9B1180615D4B4
S1136830980602D500F072F803E058061CD500F063
S113684060F80700079804900698039014D1F38821
S1136850039A00212046FEF7C6FF45E0980602D5BC
S113686000F05CF803E0580606D500F04AF8074645
S1136870079804900698039004A8019000232AE046
S11368809DF80800032808D174785CF8244004AB10
S113689003AA31464046A04724E0686800281CBF8C
S11368A0F08800281FD0307801061CD4810606D554
S11368B000F01DF801212046FFF78BF807E04006A1
S11368C006D500F014F80F212046FFF7B9F8074663
S11368D004A80190012303A800903A4631462046BB
S11368E0FFF736FF074638460AB0BDE8F08128684E
S11368F00690059600208DF8200005AA6868079088
S1136900704700200690059601208DF8200005AA06
S1136910F08807900F212046FFF792B800200690D8
S1136920059601208DF8200005AAF0880790012122
S11369302046FFF74EB830B585B00446144802909F
S1136940039101208DF8040002AA00208DF80300B1
S1136950694680208DF802004020ADF800002046F2
S1136960FEF74EFF050010D100208DF8020002AAA8
S113697069462046FEF744FF050005D080212046E5
S1136980FEF75BFF284600E0002005B030BD0000A4
S1136990FB62FF1F515FFF1FD95FFF1F0000000054
S11369A0D95FFF1F000000007B60FF1FBF60FF1F57
S11369B0000000006B61FF1FA761FF1FFB61FF1F49
S11369C02762FF1F5B62FF1F0029817814BF41F01B
S11369D0800101F07F018170704700209AE001205E
S11369E098E040686549405C70476449CA6842B1B0
S11369F08A6813780370501C8860C868401EC86099
S1136A0070470021017070475C49896908475A281A
S1136A1006D15A4A01238B54594951619169084757
S1136A207047FEB5554D0446A9616068A26802210D
S1136A30904766680FF2581050F826706846FEF7C3
S1136A408CFA1020ADF8060069464E48806800694B
S1136A5090F87900FF2818BFADF806003846FEF715
S1136A6031FA01213846FFF7AFFF40213846FEF7DF
S1136A700FFAFBF70CFE4FF47A71B0FBF1F04249C8
S1136A80B1FBF0F0002100E011464A1C00FB02F3C8
S1136A90322BF9D321B9B0F5FA7F04D8012102E0F1
S1136AA0202928BF1F21B87900F0F0000843B871ED
S1136AB001213046FEF716F8344868610120616808
S1136AC0491908710020FEBD70B505462B4C686855
S1136AD001190979A9B10FF2B80151F82060002118
S1136AE0FEF700F800213046FFF76EFF3046FEF750
S1136AF025FA6868AA680021904769680919002086
S1136B00087170BD1D488160C260C1680029FCD154
S1136B100020704738B505460FF2740050F8254040
S1136B202046FEF7C2F900F01201E17000F05001B6
S1136B30102911D04106114A14D54007A0780CD56C
S1136B4040F01000A07000208DF800006846116924
S1136B5088479DF80000207131BD00F0EF00A0705F
S1136B60207931BDA178C90603D5C007EBD5A0783B
S1136B70F3E7207952692946904731BDB08FFF1F52
S1136B805165FF1F188FFF1F40420F005765FF1FFD
S1136B90006006400070064000600E4000700E4029
S1136BA07FB50646694674682046FBF7DDFD98BB51
S1136BB00FF2481050F8245001A8FEF79BFA0098F1
S1136BC001902046FBF780FD024601A92846FEF706
S1136BD0E9F9F0B9B2680221204690470121204624
S1136BE0FDF798FF4FF400112846FEF78EFAA868C7
S1136BF040F48020A860A86840F40020A8605A20CF
S1136C00384DA9688847A968A6208847012060559F
S1136C1003E02046FBF78EFD002004B070BD10B5E4
S1136C200446304881606068A2680121904760682A
S1136C30FBF780FD002010BD38B50446294865687F
S1136C40285C48B100212846FDF764FF0FF2AC0030
S1136C5050F82500FEF72EFA2846FBF783FDA268BC
S1136C602846BDE838400021104780B50FF28C0358
S1136C70406853F82000FEF761FA002002BD10B509
S1136C80194C00F01BF8800200D508E010BD10B5C7
S1136C90164C00F013F8800200D500E010BD114935
S1136CA0E0688968BDE81040C0B2084710B5104CD0
S1136CB000F004F8800200D5F1E710BD2046FEF78D
S1136CC036BA10B50B4CFFF7F9FF800200D5E6E7A2
S1136CD010BD10B5084CFFF7F1FF800200D5DEE7C8
S1136CE010BD0000F09AFF1F00400C4000500C4003
S1136CF000600C4000700C4000600D4000400C40EF
S1136D0000500C4000600C4000700C4000600D40CE
S1136D1010B50B46DFF8B444114601205B1E22680F
S1136D20062B2ED8DFE803F0040A1519222D2C00B7
S1136D3039B30868400A00F0CAF804E009B30868E7
S1136D40400A00F08AF8E0B12268012182F859145F
S1136D5010BDB1B158328A6010BD91B102F1580032
S1136D608860BDE810400868400AB0E04FF4004075
S1136D70086001224FF4007048600A748860C8609B
S1136D80002010BD0020704770B5DFF8404420603B
S1136D90583000F070F9256805F1580000F016FB32
S1136DA006464FF4846105F15400FBF717FB206895
S1136DB00021C0F860644165002070BDDFF80C1448
S1136DC00860002009680865704738B5DFF8FC439F
S1136DD0206890F85C0430B9FCF757FE2068012164
S1136DE080F85C144165206890F85D04A0B32168C4
S1136DF0022081F85C0400F0CBF80500F7D020688D
S1136E0000F25C40C168002904BF0178022903D163
S1136E10032000F0E6F801E00121417042F27D70A8
S1136E20854219D0206800F25D400021017042F2D1
S1136E3074718D4202D10221C17431BD42F21271CA
S1136E408D4203D10221C174032002E00321C174E5
S1136E500020BDE83240C4E031BD70B50446B4F54D
S1136E60847F82B00D4630D3D84E306800F25B4147
S1136E700A7862B9887808B10F2076BDA868694697
S1136E8000F074F808B3009800F097F803E0D0F825
S1136E906404844219D130686A6800F264414B6822
S1136EA0934238BF1A468E6896199B1A641C8E60EA
S1136EB04B600C6013B9002180F85B1400F5167068
S1136EC0A968FBF78FFAFFF780FF002076BD38B57D
S1136ED00C4605466168A068FDF792FD0FF29840E4
S1136EE000E00C30416831B10268AA42F9D18268ED
S1136EF0A068FBF777FA0FF2043045B140F20111B4
S1136F006D1A0DD06D1F19D06D1E1BD027E0A1681E
S1136F10552081F8FE01AA20A16881F8FF011EE036
S1136F20A16801F5BE7400F01CF80A682260097CAF
S1136F3050F8210000F04AFA206210E0A06800F046
S1136F409AF80CE000F00DF8097C50F8215028461E
S1136F5000F03CFA0246A0682946FBF743FA0020F9
S1136F6032BD9A49096801F58C6170474269984BB2
S1136F709A4202BF426B974B9A4204BF027E012A97
S1136F8004D1C069000108600120704700207047E7
S1136F908E480068D0F86C24B2F5007F04D211004A
S1136FA004D142F27D7070474FF40071521AC0F858
S1136FB06C2400F51670FCF7AABD8449096801F237
S1136FC05A4201231370537001F58D6100239370AD
S1136FD00123D3700023137108604B6001200872F1
S1136FE070477A49096801F25A420123137090707C
S1136FF0002301F58D605370D37013710121436038
S113700003600172704730B53022027078224270FA
S1137010002282720FF2D0139400C4F11C0421FAEE
S113702004F505F00F041518E45CAC70521C082A32
S1137030F2D330BD10B5002261B10A23B1FBF3F3E2
S11370400A2404FB131130311154521C194600292F
S1137050F3D102E0302101700122002111541118F2
S1137060491E05E00A78037801F8013900F8012B7C
S11370708842F7D310BD70B504465748C0B0806845
S11370800569286814904FF6FF70B5F87A60864257
S1137090524808BF41F28836016826A8FFF7B3FFBB
S11370A055F8101F0DF1A300FFF7ADFF28686968BC
S11370B00818411E0DF1AE00FFF7A5FF69690DF137
S11370C0B900FFF7A0FF6869A9690818411E31A833
S11370D0FFF799FFA96C0DF1CF00FFF794FFE96C5E
S11370E00DF1DA00FFF78FFF296D0DF1E500FFF7D1
S11370F08AFF696D3CA8FFF786FF696815A8FFF74A
S113710099FFA9680DF15F00FFF794FF29690DF15C
S11371106A00FFF78FFFA9690DF17500FFF78AFF79
S1137120314620A8FFF786FF2D4801680DF18B003A
S1137130FFF780FFAA6D2B4B22A023A19A420CBF1C
S11371400A4602462B6A03B108460F900DF18B03E1
S11371503CA80E9013930DF1E5000D9020AB0DF1BA
S1137160DA000C9012930DF1CF000B90119231A81C
S11371700A9010910DF1B90009900DF17500089075
S11371800DF16A0007900DF15F0006900DF1AE005D
S113719005900DF1A300049015A8039026A8029071
S11371A09DF850009DF852309DF853200FF25C0179
S11371B001909DF851000090204600F023F940B062
S11371C070BD00006E6F000079657300049BFF1FA3
S11371D053544D507367746C188FFF1F2480044000
S11371E05C90FF1F6B63666730313233343536375A
S11371F0383961626364656600000000E406FF1FBD
S1137200EC06FF1FFC06FF1F0807FF1F4B696E6596
S113721074697320426F6F746C6F616465722025AA
S11372206325642E25642E25640D0A0D0A53797393
S113723074656D206465766963652049443A202548
S1137240730D0A466C6173682073697A653A202568
S1137250732062797465730D0A466C6173682072D9
S1137260616E67653A2025732D25730D0A466C619E
S1137270736820736563746F722073697A653A204A
S113728025732062797465730D0A466C61736820F6
S1137290626C6F636B733A2025730D0A52414D2063
S11372A073697A653A2025732062797465730D0ACF
S11372B052414D2072616E67653A2025732D257306
S11372C00D0A526573657276656420726567696F2D
S11372D06E20303A2025732D25730D0A526573658F
S11372E07276656420726567696F6E20313A202575
S11372F0732D25730D0A5665726966792077726954
S11373007465733A2025730D0A436865636B2072B4
S11373106573657276656420726567696F6E733A2A
S11373202025730D0A426F6F7420636F6E66696760
S11373302070726573656E743A2025730D0A50656A
S1137340726970686572616C2064657465637469E0
S11373506F6E2074696D656F75743A202573206DA6
S1137360730D0A43505520636C6F636B3A20257389
S113737020487A0D0A000000000000001407FF1FD7
S113738036000000010000004C07FF1F0E00000043
S1137390010100005C07FF1FA001000003010000C1
S11373A0FC08FF1F6000000004010000AC09FF1F7F
S11373B0A0000000050100005C09FF1F4D00000053
S11373C000000000000000000000000000F10103C4
S11373D0810704D010F8011B89B18107FAD1026832
S11373E0B2F10131914311F0803F04BF50F8042FF2
S11373F0F6E710F8011B11B110F8011BFBE7C01AE6
S1137400704700000CB41CB5044604A801900A4659
S1137410009401AB694607487844183000F018F826
S1137420009A0021117000285CBF0098001B16BC54
S11374305DF80CFB3BABFFFF70B504461E0008462D
S1137440154604D015F8011BA047761EFAD170BD6D
S11374502DE9F04784B08246894614461F46E84623
S113746007E00123224649465046FFF7E5FF8146DF
S1137470641C207810B904B0BDE8F0872528F0D149
S11374806078A41C2528014618D058285CD06328AD
S11374900ED0642818BF692814D06F2854D07028DF
S11374A058D073285DD0752818BF78284CD0E0E7F1
S11374B03868386050F8041B3860C9B24846D04771
S11374C08146D6E73868386050F8045B3860002D90
S11374D003D52D214846D047814664206F2808BF34
S11374E0082205D040F02001782914BF0A22102276
S11374F00B216428AC4603D1002D48BFCCF1000C0D
S1137500BCFBF2F502FB15CC0CF130065FFA86FCED
S11375104B1EBCF13A0FA4BFA0F15106B44403F8CA
S113752008C019465FEA050C01D00129E8DA68466B
S11375300D184846D1F10B09C2D015F8011BD047EC
S1137540B9F10109F9D1BBE73968396051F8045B35
S11375503960C3E73868386050F8045B38607820D5
S1137560BCE73868386050F8045B38602846FFF799
S11375702DFF06004846A3D015F8011BD047761E00
S1137580FAD19DE710B5BA488068006900F1680433
S113759034214FF47070F9F7AFFE48B934224FF438
S11375A070712046FAF72EFF2068B249884204D051
S11375B0FF2234212046FBF79FF8FBF79BF80020BD
S11375C010BD38B5AA4DA86804694B20E07004F1D9
S11375D010020220A070042100206070207050204E
S11375E0E0710120A07102206071002020715420FC
S11375F0E0720120A07200206072207201202063DA
S11376009D48606305F120002B69DB6A98472B696C
S1137610DB6A04F11402012100F05AF82B69DB6AD9
S113762004F11802002100F053F82B69DB6A04F11D
S11376301C02022100F04CF82B69DB6A04F12002E1
S1137640032100F045F82B69DB6A04F144020521AB
S113765000F03EF82B69DB6A04F14802062100F0D1
S113766037F82B69DB6A04F14C02072100F030F88B
S113767068680168A165E165002280492166804946
S113768061666969E26007E094F878501D4202D0AF
S1137690E5682B43E360521C182303FB02131B68A9
S11376A0002BF1D177490A6822644A68E263896849
S11376B0A16350F8101F616241680068081A401CF9
S11376C0A06201202065F9F70DFE6065002032BD3F
S11376D005F12000184700002DE9F8431546644AD7
S11376E0694C884691680427401E0E6918289946FB
S11376F05BD8DFE800F00D17191B1D1F255A5A2708
S113770029305A21233336424547494B4D4F5100C6
S1137710B9F1000F18BFC9F8007005B12E60002040
S1137720BDE8F2830C36F3E71036F1E71436EFE7E1
S11377301836EDE72036EBE72436E9E72836E7E7A5
S11377403436E5E73036E3E7D0694169496988476B
S113775020602646DCE710275836D9E74B480068F6
S1137760F6E702F1200012699269694690479DF894
S113777000000028ECD00120EAE70C273836C7E7E0
S11377804436C5E74836C3E74C36C1E75036BFE751
S11377905436BDE70836BBE79C363146404600F018
S11377A02FF80028BCD11827B2E742F63C00B7E70F
S11377B02F4A92681369401E062842F63E0219D9E0
S11377C009380BD0401E012884BFC01E032811D9DC
S11377D0083809D0401E02280CD90EE0002918BF31
S11377E0012903D119637047032901D31046704757
S11377F01965704742F63D00704742F63C007047F9
S1137800F0B589B00C46224D00E008352DB1696809
S113781000291CBF29688142F7D16A68100008BF9B
S1137820042023D06946002090470098F0B903AEA5
S1137830029001270020019001A96A683846904708
S113784040B901983060012102987A1E91400843A2
S1137850029001E000203060361D7F1C062FE9D322
S1137860182202A92046FAF7CDFD002009B0F0BD88
S1137870188FFF1F6B636667DFEF01000000FF1FB7
S1137880B7B7FF1F58800440D49BFF1F24800440D7
S11378907406FF1FAF49D1F88820531C5218C1F851
S11378A0883082F82000D1F8880000F03F00C1F849
S11378B08800704700207047B8E02DE9FC410C00B7
S11378C0154614BF002D0420984628D0A14F00204F
S11378D007F190062860707000F0A8F818B11EE057
S11378E0A22000F075F820213846FAF777FD4246C9
S11378F03946684600F0F8F810B1002129600EE01E
S11379003946684600F042F9BDF804108142E7D1D7
S1137910012030702760BDF8020028600020BDE817
S1137920F6812DE9F0410C0082B015461E4635D093
S1137930212D33D200F07AF800283FD1DFF81482E9
S113794098F8910010B1002088F8910008F16007C0
S11379505A203870A42078700EB1A52078707D80EC
S11379602DB12A46214608F16600FAF73BFD08F1DD
S11379706601384600F00AF9B880A91D384600F0BF
S113798064F8D8B9684600F0EFF8B8B99DF801007A
S1137990A12812D0A22806D0A32801D004200DE0EB
S11379A042F212700AE07888811D384600F04DF8E2
S11379B020B99DF80100A228E4D00020BDE8F6819A
S11379C065480121817000210170704720207047B3
S11379D080B55A218DF800108DF8010001205D4911
S11379E081F891000221684600F02FF802BD10B51D
S11379F00446594882B001784278807811400142A7
S1137A0011D10FF2B8100088ADF8000002222369EA
S1137A105B6869462046984723690FF2A4115B68A6
S1137A2008222046984742F2137016BD4A4801784E
S1137A3019B100210170A12004E0817819B100215D
S1137A408170A320C4E700207047444AD3690A46E2
S1137A50014618461B695B6818472DE9F14F8B46B0
S1137A601646FAF729FD04464FF47A7088467043A7
S1137A70FAF72CFDDFF8DCA00027064689460AF158
S1137A8088050EE06868296888420CD05044009943
S1137A9090F8200078547F1C6868401C00F03F0078
S1137AA068605F451DD0FAF707FD021B61EB080310
S1137AB041450AD828BFA04207D2E2436FEA08032F
S1137AC010185941421C41F10003B9F1000F08BFDD
S1137AD0002ED7D04B45D5D301D8B242D2D30520FE
S1137AE000E00020BDE8F28F70B582B005460C4678
S1137AF0164600F039F858BB6878A62804D1174810
S1137B00C069FFF774FF76BDA42106B1A5218842A0
S1137B1001D0012076BD00F023F8BDF80010698083
S1137B20B0B908462128A8BF2020688000F018F8C2
S1137B30BDF80010A98058B9698849B12046FCF7FE
S1137B405FFF69880A2000FB01F22046FFF785FFEA
S1137B5076BD000098A2FF1F28A3FF1F188FFF1FE8
S1137B6014220221684678E710B504460022012158
S1137B702046FFF772FF40B920785A28F6D1601CDE
S1137B80BDE810400A22012167E710BD30B583B07B
S1137B9004460D46684600F017F80422214668465C
S1137BA000F015F862882946684600F010F801A92B
S1137BB0684600F023F8BDF804003EBD5AA7000053
S1137BC0000201500000AAEA00210180704770B54C
S1137BD0038800240EE0655C83EA052308255E0023
S1137BE01B0444BF86F4805686F021066D1E33467E
S1137BF0F5D1641C9442EED3038070BD00880880E4
S1137C007047000005484CF22051C1814DF62811FF
S1137C10C1814FF4E9710180704700BF0020054025
S1137C2005207047087A18B9184808604C2006E007
S1137C3005207047052070471548086012204860E9
S1137C4000207047087A18B9124808604020F6E707
S1137C500520704710B5887A0F4A10B91368506828
S1137C600FE092680B891489A34202D1042800DA38
S1137C7001D1052010BD1368526853F8203052F822
S1137C80200048600B60002010BD0000C890FF1F5A
S1137C901491FF1F2891FF1F6C92FF1F00210160A8
S1137CA04160FB30417001700020704710B50446FC
S1137CB004F15800811C00220A708A72CA7204F10D
S1137CC030010A6840F8142F0A79D2094275C8793C
S1137CD098B303282CD004283ED012281ED015288F
S1137CE049D01A2842D01B2859D01D284DD01E280F
S1137CF02DD0232844D0252833D0282813D02A284F
S1137D0020D02F2846D0552835D05A282ED09E284A
S1137D1027D0A82807D0AA2814D045E02046BDE8DB
S1137D20104000F03CBD2046BDE8104000F049BDC5
S1137D302046BDE8104000F027BD2046BDE81040B5
S1137D4000F08ABD2046BDE8104000F04ABD204640
S1137D50BDE8104000F06ABE2046BDE8104000F0C7
S1137D6040BE2046BDE8104000F0C3BD2046BDE83B
S1137D70104000F07EBD2046BDE8104000F093BDE9
S1137D802046BDE8104000F0C9BD2046BDE81040C3
S1137D9000F072BE2046BDE8104000F05EBD2046F3
S1137DA0BDE8104000F069BE204600F08CFE04F1EE
S1137DB0EC0100220A704A70CA708A700A72CA7191
S1137DC010BD2DE9F0410C4684B0154662682F1DA4
S1137DD012F1010F4FF00108284605F1ED0618D104
S1137DE0317800291EBF39680968002965D095F8E3
S1137DF03710282918BFA8295FD1002101916A46AC
S1137E00216802910021009101213B681B68984779
S1137E1053E0BB68934224BF9A1ABA60B279012A2C
S1137E2009D10020B07186F801803070317B286858
S1137E30FDF71BFD41E03278002A02BF62680D2A7B
S1137E402168327852B339680968002935D06168ED
S1137E50019121680291F968009195F83710282959
S1137E6018BFA82904D13B681B686A4601219847BA
S1137E70B86848B1F86861680818F860284600F0E6
S1137E801AFB8046B868C0B9002030700D23317BDE
S1137E90286805F14802FDF7A1FC0EE060680D2892
S1137EA002BF0868DFF8D813884206D186F8038039
S1137EB0717B00F0FAFA86F808804046D0E02DE99C
S1137EC0F0410C4684B090466268002612F1010F1E
S1137ED008F1340108F1EC07404608F1040515D116
S1137EE07A78002A1EBF2A681268002A0DD0C97841
S1137EF02A2918BFAA2908D101966A462168009642
S1137F00029102212B681B689847A8E0AB68934252
S1137F1024BF9A1AAA603A7A012A07D10120F8707C
S1137F203E723E707E7200F09EF898E03A780AB392
S1137F306268019222680292EA6800922A681368D1
S1137F401A0011D0C9782A2918BFAA2902D16A4671
S1137F5002219847A86850B1E86861680818E86089
S1137F60404600F0D7FA0646A868002877D10020DA
S1137F7038705EE03879002866D060681F2802BF38
S1137F80686AC04A90425FD14A78F020024202BF38
S1137F908B78E024234257D1387B401C824253DA49
S1137FA0002B51D0112B4FDA7E72AE60CE61B448F3
S1137FB04861A86A88613E71E86AE8620A78120634
S1137FC002D410B1012000E00020387008780006C7
S1137FD003D5E86A10B1012000E0002078707878B9
S1137FE000281EBFB8780028012039D14046FFF789
S1137FF05DFE0646052E14D13878012806D1F8789E
S113800008B9012038720020387008E07878012817
S113801005D1B87808B90120F871002078700220E1
S1138020F8723878002804BF7878002817D1F879D6
S1138030A8B9797BD8F800000D2308F14802FDF7B0
S1138040CDFB0120B8720AE000F00DF8797B00F056
S11380500BF801203E71F870B870F87278713046F0
S113806004B0BDE8F081B97BD8F80000FDF7FDBB92
S11380702DE9FF47044604F1EC0660688068317C12
S1138080427900258A424FF0010A22D3006800B3E6
S113809000EBC1000838002100E0491C027891423D
S11380A017DA42680C2303FB01221378082BF4D15E
S11380B096F80FC0002000E0401C117A884205DACF
S11380C0516803015F5C6745F6D15D18D078707420
S11380D00DB901204EE0A5604FF000096A4FDFF8AA
S11380E0AC8108E0039402AA20686946FDF788FB86
S11380F0824609F10109287981451CDA00208DF8AE
S11381000400A86810F829008DF80200A96801EBA2
S113811089014988ADF80010A96801EB8901497803
S11381208DF80310C109012907BF7073CDF80880C9
S1138130B0730297D6E7002030707070F070B070A2
S11381403072F071012030710020E0607071B07104
S1138150F072707A012803D1B17B2068FDF746FBE9
S1138160B17B20681F2304F12802FDF73CFB0120AA
S11381707072504604B0BDE8F08738B5044601205B
S1138180A16861B1002506E0886810F82510206810
S1138190FDF753FB6D1CA1680A799542F4DB32BDEF
S11381A02DE9F0413A4D86B00F462968144609B1CD
S11381B0022062E02946FDF700FC060004D02846B0
S11381C0FFF76CFD304658E0286820B92846FFF7D1
S11381D065FD032051E06F60002005F1F507F8719B
S11381E0FF206B68B8712E461B686A46052130462D
S11381F098478046019800281CBF0099002938D070
S11382009DF81010009AF9706A61491EF970702285
S113821002992962A861039969620021E96105F163
S113822058010A700A22CA7100228A708A816A6916
S1138230521E02F47F431B02150A43EA026305F44B
S11382407F452B43050A05F47F4543EA126200F497
S11382507F431B0243EA00632B4343EA1060086335
S1138260C863CA6200208A6338707870266040460A
S113827003E02846FFF712FD012006B0BDE8F081B7
S11382805553425355534243077AFF1F0B79FF1F3F
S11382901C98FF1F38B5040001D1032032BDFFF73D
S11382A06CFF05462046FFF7F9FC284632BD000066
S11382B02DE9F8430546160014BF002D03204FF0A6
S11382C0010800F0EA802C1D491E052905F1EE077E
S11382D006D8DFE801F0A80306162D500020B87375
S11382E0DAE0206800281EBFB87B31788142F7D0DD
S11382F010B12846FFF741FF3078B8730020787337
S113830011E020680028EBD03088F97B0646000491
S1138310B1EB106F0BD1787BF6B2864207D02846BA
S1138320FFF72BFF7E732846FFF7A2FE8046B3E0DB
S1138330206800281CBF60680028F8D04FF00009AE
S1138340606801798945F2DA00F0A9F810D138782B
S113835028B92868FDF789FA8046012038707878B2
S113836030B931782868FDF780FA804600203870EB
S113837009F10109E4E7206800281FBF60680028AC
S1138380F8780128D3D04FF0000917E000F087F8FF
S113839012D13878012805D12868FDF770FA804693
S11383A0002038707878012806D131782868FDF7E4
S11383B066FA80460020387009F101096068017985
S11383C08945E3DB787A032818BF022813D138796A
S11383D0012813D0387A012803D1F97A2868FDF7E7
S11383E005FAF97A28680D2305F14802FDF7F6F934
S11383F0002038727872387901284DD138780028F5
S113840004BF7878002847D13871387A012803D11D
S1138410F97A2868FDF7EAF9397B00F046F800207C
S11384203872787238E03168087800F01F02012A47
S113843001BFFA7B8B88DCB294422DD14C78FE2CA0
S113844002D0FF2C11D027E0934204BF4A88002AAF
S113845020D1C98802291DDA00061BD505F1F800D0
S113846070603068C088B06016E0934204BF4A88E8
S1138470002A0FD1C98869B900060BD42846FFF732
S11384807CFE2846FFF7F4FD80460020F8700120AA
S1138490387101E04FF005084046BDE8F28380687A
S11384A0317810F829008142704728681F2305F1AC
S11384B02802FDF798B93EB500F061F8206AB0F1E2
S11384C0011F28BF4FF4803001900199E068814278
S11384D038BF084602950190042163681B68204652
S11384E0984700F046F804F1ED0007D2017B019BA8
S11384F0029A2068FDF772F9054609E001214170EE
S11385008571022181720570017B2068FDF7ADF948
S113851028463EBD3EB500F032F8606AB0F1011F56
S113852028BF4FF4803001900199E068814238BF40
S1138530084602950190032163681B68204698470A
S113854000F017F804F1EC0007D2817B019B029A3A
S11385502068FDF748F9054609E00121C17005725C
S11385600221C1720570817B2068FDF77EF92846DF
S11385703EBD6269A36921695A439142704704462A
S11385800025206900906A46704710B553688469D5
S11385906343C360126883695A430261012904BFBB
S11385A0BDE81040FFF787BFBDE81040B2E7000008
S11385B02DE9F041044604F16C050020296804F11A
S11385C0580829B921656968002900D002219CE076
S11385D0687D0028686808F1020704F1EF0640D0BE
S11385E020B9216500F0CAF878B961E0AA7D002AB3
S11385F02ED088420DD200F09CF802D100F093F8FE
S113860001E000F0BBF8002852D000F086F81120F9
S113861053E0814209D100F092F802D100F083F8CE
S113862001E000F0ABF860B96EE000F08EF804D120
S113863000F098F800F079F801E000F0A0F80028C4
S11386405CD0012184F8541003213970112161E0B8
S11386502165AA68B17A20680023FDF7BFF80220DB
S113866026E048B9F17A2068FDF7FFF8286820650C
S1138670012084F854000BE0AA7D5AB1F17A2068F5
S1138680FDF7F3F828682065022084F854000120DF
S1138690307013E0884213D200F04BF805D105F195
S11386A00C02002100F042F801E000F055F810B986
S11386B084F8540002E000F030F8B87205202AE093
S11386C081420FD100F03BF805D105F10C020021E5
S11386D000F02CF801E000F03FF8A8B1012184F883
S11386E0541015E000F031F805D100F03BF80021FA
S11386F000F01CF801E000F030F848B998F82810B0
S1138700012908BF022100D0002184F8541002E09E
S113871003213970B972BDE8F081012084F8540056
S113872003203870704705F10C0201212046FFF741
S11387302CBF081A206598F82800012870470020EB
S1138740206598F82800012870470020206598F8D3
S113875028002B68012870476B68AA68F17A2068A2
S1138760FDF741B8A0692968B3FBF0F02861A2695C
S113877002FB1010206505F10C0270476B68AA68B3
S1138780B17A2068FDF72AB800F1580101F1180206
S1138790122313605160012300219374BCE038B5A7
S11387A000F1580101F1400200230FF23C341D5D39
S11387B09D545B1C242BFAD301F11802403124236D
S11387C068E070B500F029F8282E04D159799B7916
S11387D043EA012102E0A82E00F032F81832012306
S11387E00EE070B500F019F82A2E04D159799B795E
S11387F043EA012102E0AA2E00F022F818320023F5
S113880093742B6894604B431360D16000235360CE
S113881001231374BDE87040CAE600F13903002156
S11388205D781C782D0445EA04649D7844EA0524A7
S1138830DD782C4300F1180500F15802EE7F7047F3
S113884009D15E791979360446EA01619E79DB79AA
S113885041EA06211943704700E000BF00F15801C6
S1138860002241F8182F01228A7400224A600A74F7
S11388709EE638B500F1580101F1640200230FF2BD
S11388808C241D5D9D545B1C082BFAD301F1180246
S1138890643108235160136000210123117493741F
S11388A0BDE8324084E638B5044604F1580505F1C4
S11388B0640000210FF254228B5C0B54491C0829DC
S11388C0FAD305F11800082101600121817405F132
S11388D064014160002101742046FFF769FE94F8A9
S11388E03810C90704D5A91C05220A7024228A72EB
S11388F032BD90F8373000F15801252B01F11802F0
S113890003D1082313602C3102E00C2313603431AB
S11389105160012191740021117449E62DE9F0415F
S11389200FF2C01186B00968009100F1580890F860
S11389303F5098F86C6000210022002300F11404D9
S113894026B1A668002E14BF0226032627680197C5
S1138950D4F804E00397F400F7000C37CDF808E0EE
S11389608DF80340CDF810E0BD4288BF3D466F4608
S1138970D2B201EB0804D75D521C491C042984F8C7
S11389806D70F4D3002203AFC9B2D75D01EB0804C4
S1138990521C491C082A84F86D70F4D398F86C2092
S11389A08AB100220CE001AFDBB201EB0804DF5D09
S11389B084F86D705B1C491CC9B20829F3D3521C9E
S11389C0D2B2B242F8DB012208F118018A7408F12C
S11389D06D024A600D6000220A7406B0BDE8F041E1
S11389E0E6E538B5054605F1580404F11800002100
S11389F00160012181740021416001742846FFF760
S1138A00D7FD05F138010A7F022A0ED00A7802F058
S1138A101F02172A02D100220A7732BD01220A77E7
S1138A20A11C05220A7024228A7232BD2DE9F0416C
S1138A30044604F13B0604F15805377805F11800A3
S1138A400021016000F038F88046707E022808D0CA
S1138A50F80706D5012070760521A81C0170242191
S1138A60817260680368180003D000220721204641
S1138A7098474046BDE8F081F0E670B582B0044600
S1138A8004F13B0504F15800297801F003018DF845
S1138A900010002140F8181F00F00EF80646687E0A
S1138AA0022807D060680368180003D06A460821CA
S1138AB020469847304676BD0121817400214160EB
S1138AC00174204674E500F15801002240F8502F4B
S1138AD00122027105208870202008730020487349
S1138AE07047000000000000008004022000000025
S1138AF046534C2053454D4946534C204D41535306
S1138B002053544F5241474530303031000000006B
S1138B1000000000DFF8D8130A7B01F25A4100205C
S1138B200B7803B10120DFF8CC331A705870C97F79
S1138B30002914BF104300207047000070B50024C2
S1138B40491E1546DFF8A833112903F1080603F27C
S1138B5079425CD8DFE801F0095B5B5B5B5B0B1A75
S1138B603D42474C51565B5B292E14704FE0002D5B
S1138B704DD0012010702878507029783068FCF7A7
S1138B8058FB2978B06CFEF7FDF840E01078002817
S1138B903DD02A88110A022939DAC81880F87B24C2
S1138BA0D2B23068FCF759FB31E0002D2FD0507859
S1138BB028702CE05DB32A88100A022807DAC0184E
S1138BC002F47F4190F87B04084328801FE00524C9
S1138BD01DE0E5B12946FFF72FF817E0BDB129469E
S1138BE0FFF730F812E095B12946FFF733F80DE0AE
S1138BF06DB12946FFF714F808E045B12946FFF79F
S1138C0011F803E01DB12946FFF714F80446204685
S1138C1070BDF8B50FF21030B54C0078B64E8DF833
S1138C20000005464FF490612046F9F7D7FBF9F7A9
S1138C3015FD0028B06800690CD190F8781001F097
S1138C40EF0180F87810B0680069C16821F0100164
S1138C50C1602DE000F17C064FF6FF717288308808
S1138C608A4208BF884209D0A44908723088000AA1
S1138C704872708888727088000AC8727068A04F41
S1138C8010F1010F04D01021F8F736FB00B9776812
S1138C909C489D4E076004F58F60002101800020F0
S1138CA0A0602065206022463146FCF7E5FE08B14D
S1138CB00120F2BD3068006920652046FEF764F8A3
S1138CC030684068A0602046FCF7D5FA68B201001D
S1138CD007D58E4A01F00F039A18402002F8040CBD
S1138CE002E08B4B4022C254012005F01F02904049
S1138CF0884A490942F821002068FCF75BFD0020FE
S1138D00F2BD10B50020FCF713FFA0B9784C204643
S1138D10FEF754F82046FCF7B2FA7F48016849038D
S1138D2009D57E4A4FF4001111607D4A1160016833
S1138D3021F48021016010BD38B56E4C794D0020BE
S1138D40207001206070FBF7E6F8FEF73EF8A87883
S1138D50032803D10020A870FAF70EFFFBF7E1F80F
S1138D60287800B1012060700120207031BD10B559
S1138D705F4C002104F11400FBF7B2F8002104F168
S1138D801800FBF7ADF804F11400FBF7B5F8002068
S1138D9010BD2DE9F0410C00154614BF002D042030
S1138DA039D00020286013B1012B02D02CE0012619
S1138DB000E002264F48007860B3DFF8348108F100
S1138DC00807B87930B13868242308F12002022159
S1138DD0FCF707FC0120B8714FF0FF3108F11400D3
S1138DE0FBF780F8387EB04206D0012E08BF022877
S1138DF00AD142F212700EE0B87EF97E40EA0120F8
S1138E007969091F814201D2012004E008F124019B
S1138E10216028600020BDE8F0812DE9F04135484B
S1138E20007800280C4615463ED0212D28BF04208A
S1138E303BD213B1012B10D011E00327DFF8B0802F
S1138E40FBF769F808F10806707950B100207071D9
S1138E50FBF767F842F2127027E00427EEE70120DF
S1138E6023E0FBF75EF8377600207076B576280AA3
S1138E70F076002C18BF002D05D02A46214608F1B3
S1138E802400F9F7AFFA98F8460001280CD13068AD
S1138E90242308F120020121FCF793FB4FF0FF315A
S1138EA008F11800FBF71EF80020BDE8F08110B5AA
S1138EB04469A468002300220021A04710BD0020BB
S1138EC070472020704710B5094C94F85C040228C0
S1138ED018BF032807D104F11400FBF711F804F1BB
S1138EE01800FBF70DF82068BDE81040FDF74ABAFA
S1138EF030A3FF1FB0A7FF1F188FFF1F1491FF1F80
S1138F006C92FF1F2CA3FF1F888FFF1F18ED00E03A
S1138F1000E400E000E100E03480044084E100E08B
S1138F2084E200E08AA7FF1F3500000000F00BF880
S1138F30002801D000F00AF80020C046C046FAF725
S1138F40B4FFFAF7CBFF01207047000010B50749C2
S1138F5079441831064C7C44163404E00A68081D30
S1138F60511888470146A142F8D110BD3C040000C5
S1138F70500400002925FF1F3725FF1FEC04FF1FA5
S1138F808099FF1FCC06FF1FCC8FFF1FDC0AFF1F39
S1138F90088FFF1F7C05FF1F640AFF1FD405FF1FF6
S1138FA000000000000000000000000000000000BD
S1138FB000000000000000000000000000000000AD
S1138FC0000000000000000000000000000000009D
S1138FD0000000000000000095010000C94CFF1FC4
S1138FE0000000009490FF1F5968FF1F000000005C
S1138FF0C090FF1F708FFF1F8586FF1F02000000B7
S1139000000000000000000000000000000000005C
S11390109946FF1FB746FF1F000000000000000034
S11390200000000000000000000000003365FF1F86
S11390305765FF1F0000000000000000FFFF030051
S1139040010000008406FF1F0000FF1FFFFF022035
S1139050010000004C0AFF1F00000068FFFFFF6FC3
S113906000000000F00AFF1F00000004FFFFFF07DC
S113907000000000080BFF1F00000040FFFF074036
S1139080000000004406FF1F00000840FFEF0F40EF
S1139090000000004406FF1F00F00F40FFFF0F40D8
S11390A0000000004406FF1F000000E0FFFF0FE087
S11390B0000000004406FF1F000000000000000044
S11390C00000000000000000000040018103400097
S11390D0020340008302400004024000000000003C
S11390E0020000006090FF1F000000000300000069
S11390F07090FF1F01000000010000008090FF1F1E
S11391008C90FF1F0101000000000000020000001D
S11391106890FF1F00000000080650019C90FF1F8C
S11391200100000001000000AC90FF1FB890FF1F79
S1139130030100000600FF0901A1018501190129AD
S113914001150026FF007508952391028502190177
S11391502901150026FF007508952391028503193E
S1139160012901150026FF00750895238102850455
S113917019012901150026FF00750895238102C0F5
S11391801201000200000040A21573000200010257
S11391900301000009024000020100C0320904007A
S11391A0000203000003092100010001224C000712
S11391B00581034000010705020340000109040181
S11391C00002080650030705830240000007050457
S11391D002400000040309043A034600520045001B
S11391E045005300430041004C004500200053005B
S11391F045004D00490043004F004E004400550017
S1139200430054004F005200200049004E00430028
S11392102E0000002A0355005300420020004300A2
S11392204F004D0050004F005300490054004500CA
S1139230200044004500560049004300450000005A
S11392403E034D004300550020004D0053004300F1
S1139250200041004E004400200048004900440022
S11392602000470045004E004500520049004300DD
S1139270200044004500560049004300450000001A
S113928022034200410044002000530054005200D5
S113929049004E00470000000000000000000000EC
S11392A000000000040000003A0000002A00000052
S11392B03E000000220000006891FF1F6C91FF1F18
S11392C0A891FF1FD491FF1F1492FF1F4C92FF1F00
S11392D03892FF1F090400006891FF1F040000007A
S11392E06092FF1F0100000030B504E012F8014B4A
S11392F000F8014B491ED1B1C507F7D40129F5D0B7
S1139300850701D4042904D232F8024B20F8024B19
S1139310891E8B08EFD000EB830403E052F8045B52
S113932040F8045BA042F9D3A1EB8301E3E730BD2D
S113933080B513460246184600E080B5FFF7D4FF17
S1139340002002BD10B514460A462146BDE810406F
S11393500123F7F7E9BAFFF7FEBFC046C046C0468F
S1139360C046FFF7E3FD19E050F8041BCB0744BFE8
S1139370A9F101035918121F0023042A41F8043BE0
S1139380F9D25FEA827C0B4604D54FF0000CA1F8B9
S113939000C09B1CD10744BF0021197050F8042B56
S11393A0002AE1D170470000BFFFFFFF2005000045
S11393B00094FF1F940E00002099FF1F000000007E
S11393C062B38B0708D0521E11F8013B00F8013B31
S11393D000F024808B07F6D1830740F0208000BF83
S11393E0103A07D330B4B1E83810103AA0E8381076
S11393F0F9D230BC530724BFB1E80810A0E8081024
S113940044BF51F8043B40F8043BD20724BF31F871
S1139410022B20F8022B44BF0B7803707047083AE4
S113942007D3B1E80810083A40F8043B40F804CBED
S1139430F7D25307E4E7FEE780B51B491B480860F1
S11394401B491C48421A1C4888421CBF002AFFF7CB
S1139450B7FF1A481A49091A18BF00F041F8194809
S11394601949091A18BF00F03BF818491848421A5C
S113947004D0BDE808401748FFF7A2BF01BD164855
S11394804FF0FF31016041608160C1600161416161
S11394908161C1611148016041608160C160016105
S11394A041618161C161704708ED00E00000000086
S11394B0000000000000000000000000FCFD02208D
S11394C000FE022000FE022000FE0220289600007A
S11394D02896000000FE022080E100E080E200E027
S11394E0002200F001B80000401810F0030308D077
S11394F0C91A1FD3DB0748BF00F8012D28BF20F885
S1139500022D130030B414461546103928BF20E943
S11395103C00FAD8490728BF20E90C0048BF40F8AE
S1139520042D890028BF20F8022D48BF00F8012D22
S113953030BC7047C91818BF00F8012DCB0728BFED
S113954000F8012D7047000005484CF22051C181FC
S11395504DF62811C1814FF4E9710180704700BFB5
S11395600020054000F00BF8002801D000F00AF8B4
S11395700020C046C046F6F79BFF00F017F8012014
S11395807047000010B5074979441831064C7C44F3
S1139590163404E00A68081D511888470146A142A0
S11395A0F8D110BD740000008000000000F000B885
S11395B00746384600F002F8FBE7000020210903C3
S11395C026311820ABBEF9E7FFF7FEBFC046C04600
S11395D0C046C046FFF7C6FF19E050F8041BCB078E
S11395E044BFA9F101035918121F0023042A41F8AA
S11395F0043BF9D25FEA827C0B4604D54FF0000CA1
S1139600A1F800C09B1CD10744BF0021197050F879
S1139610042B002AE1D17047C1FFFFFF04000000C2
S10B9620FCFD02200000000023
S9030411E7
